:100000000CEF00F0039E000CD8CFF3F3E0CF3CF0F0
:04001000E6EF1DF00A
:1000180001EE00F013EEE7F047EC30F000EE3DF0B3
:1000280010EE40F047EC30F000EE41F011EE00F039
:1000380047EC30F000EE14F010EE3DF047EC30F0F5
:10004800A7EF1EF0FFFF04FE10FC23FA3EF860F64F
:100058008AF4BAF2F1F02FEF73EDBEEB0FEA66E81F
:10006800C3E626E58EE3FCE170E0E9DE68DDEBDB64
:1000780074DA02D994D72CD6C7D468D30DD2B7D0A6
:1000880064CF17CECDCC87CB46CA08C9CEC798C691
:1000980066C537C40CC3E5C1C1C0A0BF83BE69BD76
:1000A80052BC3FBB2FBA21B917B810B70BB60AB567
:1000B8000BB40FB316B220B12CB03BAF4CAE60AD51
:1000C80077AC8FABABAAC8A9E8A80BA82FA756A6F0
:1000D8007FA5AAA4D7A306A338A26BA1A1A0D89FE5
:1000E800119F4D9E8A9DC99C0A9C4C9B919AD799B9
:1000F8001F996998B49701975096A095F2944694E1
:100108009B93F1924992A391FE905A90B88F178FC2
:10011800788EDA8D3E8DA38C098C708BD98A438AB0
:10012800AE891B898988F8876887D9864C86BF85F8
:100138003485AA842184998312838D8208828581DB
:10014800028181800180DD000001E16BE0AF14D005
:10015800DDC000F0DEC001F0DFC002F0E0C003F057
:100168004EEC30F000C0DDF001C0DEF002C0DFF080
:1001780003C0E0F0010EE16F830E046EF90E056E08
:10018800220E066E3E0E076EDD0EE96E000EEA6E5A
:100198003CEC30F0DDC0EAF0DEC0EBF0DFC0ECF0A4
:1001A800E0C0EDF05AEC2DF000C004F001C005F0FD
:1001B80002C006F003C007F0DDC000F0DEC001F0A9
:1001C800DFC002F0E0C003F0FFEC2DF0046A056A1E
:1001D800800E066E400E076ECEEC2CF000C0DDF0EF
:1001E80001C0DEF002C0DFF003C0E0F0DDC004F0C3
:1001F800DEC005F0DFC006F0E0C007F0006A016A63
:10020800026A400E036E50EC2FF0D8B011D0046A89
:10021800056A066A400E076EDD0EE96E000EEA6E8C
:1002280006EC30F00001E151000ED8B4010EE16F88
:10023800DDC004F0DEC005F0DFC006F0E0C007F066
:10024800006A016A800E026E3F0E036E50EC2FF0BA
:10025800DDC004F0DEC005F0DFC006F0E0C007F046
:10026800D8B017D0006A016A026A400E036EFFEC2C
:100278002DF000C0DDF001C0DEF002C0DFF003C0E9
:10028800E0F0DDC004F0DEC005F0DFC006F0E0C03D
:1002980007F0DDC000F0DEC001F0DFC002F0E0C012
:1002A80003F0CEEC2CF000C0E2F001C0E3F002C095
:1002B800E4F003C0E5F0E2C0F2F0E3C0F3F0E4C01C
:1002C800F4F0E5C0F5F00001820EF66F050EF76F49
:1002D800030EF86FF96B3EEC2CF000C0E6F001C09D
:1002E800E7F002C0E8F003C0E9F0E2C0F2F0E3C0D2
:1002F800F3F0E4C0F4F0E5C0F5F000016E0EF66F1F
:10030800050EF76F040EF86FF96B3EEC2CF0E6C0A3
:1003180004F0E7C005F0E8C006F0E9C007F023ECF8
:1003280027F000C004F001C005F002C006F003C0C9
:1003380007F0DD0EE96E000EEA6E3CEC30F00001CD
:10034800E151DDC000F0DEC001F0DFC002F0E0C026
:1003580003F0D8B412004EEF30F00E6A02340334C2
:100368000C6E04E00E36036A028E1200006A016AFF
:10037800026A036A000C0E92063407340D6E05E01B
:10038800D8B00E82076A068E12000D6A046A056AE2
:10039800066A076A12000C50E9E0029E0E320C3021
:1003A800036ED8B0028ED0EF2FF00C521EE003502F
:1003B8000DE0030404E1002A012202220322D8905E
:1003C80003320232013200320C2AEFD700500110FA
:1003D800021003100AE002BEDED70C4ECCEF2FF05D
:1003E800D890003601360236F6D7CCEF2FF0A6A209
:0403F8001200FDD71B
:100400000000020001000400FF00030004000200DD
:1004100003000000FF0001000000B4420A00AE42E9
:100420002612AD42CF82AB4291C8A942CEFBA74271
:10043000E624A6427F47A4426B65A242A47FA04265
:10044000B5969E42E9AA9C4265BC9A4238CB984236
:100450005CD79642C4E0944257E79242F6EA904253
:100460007BEB8E42BDE88C428DE28A42B8D888424E
:1004700005CB864239B9844213A382424E8880421A
:100480003BD17C4264877842693274428ED16F429C
:1004900008646B42FCE86642795F62427CC65D425A
:1004A000E61C59427E615442EA924F42A9AF4A4249
:1004B00013B6454248A4404230783B426B2F364247
:1004C00042C73042993C2B42D58B2542BEB01F42D9
:1004D0005AA61942B066134286EA0C42EC2806423C
:1004E0004F2DFE41834AEF411883DF4158A2CE4190
:1004F0004B5CBC413D3CA841807D914141406D41F8
:100500001687274100000000A632943198319C31B3
:10051000A031A032A032A032A032A632A632A6323A
:10052000A632A632A632A632A632A632A6320635A8
:10053000A632A632A6322238223822382238223871
:10054000D237063C04427D9F6A425C900142604D76
:10055000BB4051EC473EDE8D1FBB063C0442C059F8
:100560008B4274044442F99B4F410000803FECF3FE
:100570004A48359595C717C1DC45FDDB6DC372B39D
:1005800033402B3401487F9DB045E7FFD94200003E
:10059000803FAF00D96E030ED926D9500001AF6F4E
:1005A000AFC004F0B0C005F0B1C006F0B2C007F0B3
:1005B000006A500E016EC30E026E470E036ECEEC43
:1005C0002CF00AEC2FF000C0B0F001C0B1F002C076
:1005D000B2F003C0B3F0FBEC01F00001AF51A96E23
:1005E000AF07B051A86E3F0EA616D890F2BED880C5
:1005F000F29EA684550EA76EAA0EA76EA682A1989B
:10060000A694D8B0F28EB1C0B0F0B2C0B1F0B3C011
:10061000B2F0B36BB2BFB307FBEC01F00001AF5116
:10062000A96EAF07B051A86E3F0EA616D890F2BEC5
:10063000D880F29EA684550EA76EAA0EA76EA6823B
:10064000A198A694D8B0F28EB1C0B0F0B2C0B1F00B
:10065000B3C0B2F0B36BB2BFB307FBEC01F0000163
:10066000AF51A96EAF07B051A86E3F0EA616D89035
:10067000F2BED880F29EA684550EA76EAA0EA76E73
:10068000A682A198A694D8B0F28EB1C0B0F0B2C044
:10069000B1F0B3C0B2F0B36BB2BFB307FBEC01F083
:1006A0000001AF51A96EB051A86E3F0EA616D890AA
:1006B000F2BED880F29EA684550EA76EAA0EA76E33
:1006C000A682A198A694D8B0F28E12000001B76F4E
:1006D000BC6BBD6BBE6BBF6BFBEC01F00001B75197
:1006E000A96EB72B3F0EA616A680A8CF00F0016A10
:1006F000026A036A0050BC130150BD130250BE13BE
:100700000350BF13BEC0BFF0BDC0BEF0BCC0BDF043
:10071000BC6BFBEC01F00001B751A96EB72B3F0E8B
:10072000A616A680A8CF00F0016A026A036A0050EC
:10073000BC130150BD130250BE130350BF13BEC003
:10074000BFF0BDC0BEF0BCC0BDF0BC6BFBEC01F0A7
:100750000001B751A96EB72B3F0EA616A680A8CFF1
:1007600000F0016A026A036A0050BC130150BD1315
:100770000250BE130350BF13BEC0BFF0BDC0BEF0D9
:10078000BCC0BDF0BC6BFBEC01F00001B751A96E21
:100790003F0EA616A680A8CF00F0016A026A036A7F
:1007A0000050BC130150BD130250BE130350BF13C1
:1007B000BCC000F0BDC001F0BEC002F0BFC003F07D
:1007C000F8EC2FF000C0B8F001C0B9F002C0BAF0E8
:1007D00003C0BBF0046A500E056EC30E066E470ED2
:1007E000076EB8C000F0B9C001F0BAC002F0BBC0DB
:1007F00003F023EF27F0CC000001CFAF0CD0046A48
:10080000056A800E066EBF0E076ECC0EE96E000EF6
:10081000EA6E3CEC30F03B0EF36EF46AF3CF00F07E
:10082000F4CF01F0D89000360136D890003601366A
:100830000050180FF66E0150F76E040EF7220900F3
:10084000F5CF04F00900F5CF05F00900F5CF06F06B
:100850000900F5CF07F0CCC000F0CDC001F0CEC04C
:1008600002F0CFC003F050EC2FF0D8B003D0F3501B
:10087000020F1200F306D8A0F406F4BE000CCED787
:100880000001420E5A6F650E596F2E0E586FE10E21
:10089000576F01010053D8A409D00001420E5A6FCE
:1008A000680E596F420E586F110E576F00013C0EC3
:1008B0005E6F8E0E5D6FFA0E5C6F350E5B6F010121
:1008C0000053D8A409D000013C0E5E6F8D0E5D6F01
:1008D000150E5C6F9E0E5B6F200EF8DE00C077F089
:1008E00001C078F002C079F003C07AF0240EEEDE89
:1008F00000C07FF001C080F002C081F003C082F030
:100900005BC004F05CC005F05DC006F05EC007F09F
:1009100077C000F078C001F079C002F07AC003F02F
:10092000CEEC2CF000C087F001C088F002C089F046
:1009300003C08AF05BC004F05CC005F05DC006F047
:100940005EC007F07FC000F080C001F081C002F0FF
:1009500082C003F0CEEC2CF000C08FF001C090F00C
:1009600002C091F003C092F00001400EA26FC00ED1
:10097000A16FA06B9F6B400EA66FC30EA56F410EBB
:10098000A46F160EA36F9FC004F0A0C005F0A1C015
:1009900006F0A2C007F077C000F078C001F079C07F
:1009A00002F07AC003F023EC27F000C0EAF001C0A7
:1009B000EBF002C0ECF003C0EDF05AEC2DF00AECC5
:1009C0002FF000C05FF001C060F0A3C004F0A4C02D
:1009D00005F0A5C006F0A6C007F077C000F078C00B
:1009E00001F079C002F07AC003F023EC27F000C0D8
:1009F000EAF001C0EBF002C0ECF003C0EDF05AECFD
:100A00002DF00AEC2FF000C061F001C062F05FC071
:100A100000F060C001F0EAEC2FF09FC004F0A0C02D
:100A200005F0A1C006F0A2C007F0CEEC2CF000C08B
:100A300004F001C005F002C006F003C007F077C063
:100A400000F078C001F079C002F07AC003F0FFEC4A
:100A50002DF09FC004F0A0C005F0A1C006F0A2C018
:100A600007F023EC27F0046A056A066A3F0E076E5A
:100A700001EC2EF000C0A7F001C0A8F002C0A9F060
:100A800003C0AAF000EE61F0EECF00F0EDCF01F070
:100A9000EAEC2FF0A3C004F0A4C005F0A5C006F056
:100AA000A6C007F0CEEC2CF000C004F001C005F0A9
:100AB00002C006F003C007F077C000F078C001F074
:100AC00079C002F07AC003F0FFEC2DF0A3C004F06F
:100AD000A4C005F0A5C006F0A6C007F023EC27F0DF
:100AE000046A056A066A3F0E076E01EC2EF000C02C
:100AF000ABF001C0ACF002C0ADF003C0AEF012002C
:100B0000B0000001B96FB851B0C000F0B1C001F041
:100B1000B2C002F0B3C003F0D8B423D004EC30F07C
:100B2000046A056A066A490E076E23EC27F000C0C6
:100B3000C4F001C0C5F002C0C6F003C0C7F0B4C025
:100B400000F0B5C001F0B6C002F0B7C003F004EC8D
:100B500030F0046A056A066A490E076E23EC27F036
:100B600022D004EC30F0046A056A066A480E076E6B
:100B700023EC27F000C0C4F001C0C5F002C0C6F0ED
:100B800003C0C7F0B4C000F0B5C001F0B6C002F0B9
:100B9000B7C003F004EC30F0046A056A066A480E38
:100BA000076E23EC27F000C0C0F001C0C1F002C006
:100BB000C2F003C0C3F0C4C004F0C5C005F0C6C095
:100BC00006F0C7C007F00001B951040DA70EF324C9
:100BD000E96E000EF420EA6EEECF00F0EECF01F0E9
:100BE000EECF02F0EECF03F0FFEC2DF000C0EAF004
:100BF00001C0EBF002C0ECF003C0EDF05AEC2DF0B8
:100C00000AEC2FF00001B951020D5F0EF324E96EDA
:100C1000000EF420EA6EEECF02F0EDCF03F00250AA
:100C20000024BA6F03500120BB6FBAC000F0BBC0F4
:100C300001F0EAEC2FF0C4C004F0C5C005F0C6C056
:100C400006F0C7C007F001EC2EF0B951040D9F0E5D
:100C5000F324E96E000EF420EA6EEECF04F0EECF3E
:100C600005F0EECF06F0EECF07F0CEEC2CF000C092
:100C700073F001C074F002C075F003C076F073C069
:100C8000CCF074C0CDF075C0CEF076C0CFF0B4DD3E
:100C9000006E0004D96E0001B951D95ED950D8A4B4
:100CA00007D0C86BC96BB40ECA6F430ECB6F1CD094
:100CB000D9CF00F0C6EC2FF000C004F001C005F061
:100CC00002C006F003C007F0006A016AB40E026EAB
:100CD000430E036E23EC27F000C0C8F001C0C9F03A
:100CE00002C0CAF003C0CBF0C8C004F0C9C005F010
:100CF000CAC006F0CBC007F07FC000F080C001F092
:100D000081C002F082C003F023EC27F000C0EAF0BB
:100D100001C0EBF002C0ECF003C0EDF05AEC2DF096
:100D20000AEC2FF000C0BEF001C0BFF0BEC000F062
:100D3000BFC001F0EAEC2FF0C8C004F0C9C005F054
:100D4000CAC006F0CBC007F0CEEC2CF000C004F017
:100D500001C005F002C006F003C007F07FC000F03C
:100D600080C001F081C002F082C003F0FFEC2DF0E2
:100D7000C8C004F0C9C005F0CAC006F0CBC007F077
:100D800023EC27F0046A056A066A3F0E076E01EC41
:100D90002EF0C0C004F0C1C005F0C2C006F0C3C050
:100DA00007F0FFEC2DF000C0EAF001C0EBF002C04C
:100DB000ECF003C0EDF05AEC2DF00AEC2FF000013E
:100DC000BE510024BC6FBF510120BD6FBCC000F0FC
:100DD000BDC001F0EAEC2FF0C0C004F0C1C005F0C6
:100DE000C2C006F0C3C007F001EC2EF0C8C004F08A
:100DF000C9C005F0CAC006F0CBC007F0CEEC2CF09D
:100E000000C07BF001C07CF002C07DF003C07EF02A
:100E100012005BC004F05CC005F05DC006F05EC06F
:100E200007F073C000F074C001F075C002F076C026
:100E300003F0CEEC2CF000C083F001C084F002C0BF
:100E400085F003C086F05BC004F05CC005F05DC0B7
:100E500006F05EC007F07BC000F07CC001F07DC0F2
:100E600002F07EC003F0CEEC2CF000C08BF001C08D
:100E70008CF002C08DF003C08EF08FC004F090C0E3
:100E800005F091C006F092C007F08BC000F08CC056
:100E900001F08DC002F08EC003F0FFEC2DF000C019
:100EA000D9F001C0DAF002C0DBF003C0DCF028ECBE
:100EB0002EF000C0B9F001C0BAF002C0BBF003C010
:100EC000BCF083C0D9F084C0DAF085C0DBF086C006
:100ED000DCF028EC2EF000C0BDF001C0BEF002C076
:100EE000BFF003C0C0F087C0D9F088C0DAF089C075
:100EF000DBF08AC0DCF028EC2EF0BDC004F0BEC0F0
:100F000005F0BFC006F0C0C007F0CEEC2CF0B9C0B1
:100F100004F0BAC005F0BBC006F0BCC007F0CEECD0
:100F20002CF000C0C1F001C0C2F002C0C3F003C089
:100F3000C4F083C0DDF084C0DEF085C0DFF086C081
:100F4000E0F0A8EC00F000C0C5F001C0C6F002C09F
:100F5000C7F003C0C8F087C0DDF088C0DEF089C0EC
:100F6000DFF08AC0E0F0A8EC00F0C5C004F0C6C015
:100F700005F0C7C006F0C8C007F0CEEC2CF0C1C029
:100F800004F0C2C005F0C3C006F0C4C007F001EC15
:100F90002EF000C0C9F001C0CAF002C0CBF003C0FF
:100FA000CCF06FEC2FF0046A180E056EC70E066EBB
:100FB000450E076ECEEC2CF000C0B5F001C0B6F0C7
:100FC00002C0B7F003C0B8F0B5C004F0B6C005F079
:100FD000B7C006F0B8C007F0006A016A7A0E026E68
:100FE000440E036ECEEC2CF00AEF2FF083C0D9F044
:100FF00084C0DAF085C0DBF086C0DCF028EC2EF08F
:1010000000C0BDF001C0BEF002C0BFF003C0C0F020
:101010008FC004F090C005F091C006F092C007F0B8
:101020008BC000F08CC001F08DC002F08EC003F0C8
:10103000FFEC2DF000C0DDF001C0DEF002C0DFF0FB
:1010400003C0E0F0A8EC00F0BDC004F0BEC005F0A5
:10105000BFC006F0C0C007F0CEEC2CF000C0D1F04D
:1010600001C0D2F002C0D3F003C0D4F08FC004F0AE
:1010700090C005F091C006F092C007F08BC000F060
:101080008CC001F08DC002F08EC003F0FFEC2DF09B
:1010900000C0D9F001C0DAF002C0DBF003C0DCF020
:1010A00028EC2EF000C0C1F001C0C2F002C0C3F0B5
:1010B00003C0C4F083C0D9F084C0DAF085C0DBF08F
:1010C00086C0DCF028EC2EF000C0C5F001C0C6F0F0
:1010D00002C0C7F003C0C8F087C0DDF088C0DEF0F2
:1010E00089C0DFF08AC0E0F0A8EC00F0C5C004F0D1
:1010F000C6C005F0C7C006F0C8C007F0CEEC2CF0A3
:10110000C1C004F0C2C005F0C3C006F0C4C007F0FF
:10111000CEEC2CF000C0C9F001C0CAF002C0CBF088
:1011200003C0CCF083C0DDF084C0DEF085C0DFF00A
:1011300086C0E0F0A8EC00F000C0CDF001C0CEF019
:1011400002C0CFF003C0D0F087C0D9F088C0DAF079
:1011500089C0DBF08AC0DCF028EC2EF0CDC004F0B2
:10116000CEC005F0CFC006F0D0C007F0CEEC2CF01A
:10117000C9C004F0CAC005F0CBC006F0CCC007F06F
:10118000FFEC2DF000C0D5F001C0D6F002C0D7F0C2
:1011900003C0D8F08FEC2BF000C0B9F001C0BAF05A
:1011A00002C0BBF003C0BCF057C004F058C005F04B
:1011B00059C006F05AC007F0B90EE96E000EEA6E8B
:1011C0003CEC30F0046A056AB40E066E430E076EFE
:1011D000B90EE96E000EEA6E08EC30F0046A056A9A
:1011E000B40E066E430E076EB9C000F0BAC001F02F
:1011F000BBC002F0BCC003F050EC2FF0D8A00CD064
:10120000046A056AB40E066E430E076EB90EE96EE7
:10121000000EEA6E06EC30F0B9C000F0BAC001F082
:10122000BBC002F0BCC003F01200E96E010EE16E1B
:10123000E950D96EE1CF01F0D9CF00F0012A02D0F8
:10124000D8900032012EFCD70050E96EE950D91A2F
:10125000020EE96001D004D0E150080AD8A402D0FF
:10126000D9501200D890E136E5D7B7001650D8A46F
:1012700002D0D8901200B7C0E9FFB8C0EAFF15C08D
:10128000EFFF166AD88012009EA8FED7AD6E9E981A
:101290001200D96E0A0ED96002D0300E01D0370E7E
:1012A000D926D950F1D7E16EE1380F0BF2DFE150CA
:1012B0000F0BEFD7B000B0C0E1FFB1C0E2FFE750C5
:1012C000D8B41200E1CFE9FFE2CFEAFFE14AE22A17
:1012D000EF50DADFF4D7B0000001B251006EB35125
:1012E000016EB207000EB35B01500010D8B41200BB
:1012F000FBEC01F00001B051A96EB04BB12B3F0ED9
:10130000A616A680A850C0DFE7D7BB00D96A0001A7
:10131000BB05BC11BD11BE11D8A40FD01FD000EE6B
:101320009BF00001BB51EE5EBC51EE5ABD51EE5A2E
:10133000BE51ED5AED52ED52D92A00EE9EF0000159
:10134000BE51ED5C08E1BD51ED5C05E1BC51ED5CC9
:1013500002E1BB51EF5CD8A003D0E1D79BC0D9FF1D
:10136000D950D8B403D0010EE8CF07F101010753DB
:10137000D8A40ED0D950D8A40BD00001BF05D8B442
:1013800034D10001BF51020AD8A41200200E7CD72C
:10139000D950300F79D7E16E0001E80EBB6F030E14
:1013A000BC6FBD6BBE6BE150BF6FB0DF640E000160
:1013B000BB6FBC6BBD6BBE6BE150BF6FA7DF0A0E8E
:1013C0000001BB6FBC6BBD6BBE6BE150BF6F9EDF9E
:1013D00090D0F36E0001A00EBB6F860EBC6F010EA5
:1013E000BD6FBE6BF350BF6F91DF0001100EBB6F7E
:1013F000270EBC6FBD6BBE6BF350BF6F87DFF35022
:10140000CAD7F46E0001BB6BCA0EBC6F9A0EBD6FDB
:101410003B0EBE6FF450BF6F79DF0001BB6BE10E76
:10142000BC6FF50EBD6F050EBE6FF450BF6F6EDF63
:101430000001800EBB6F960EBC6F980EBD6FBE6B29
:10144000F450BF6F63DF0001400EBB6F420EBC6FF4
:101450000F0EBD6FBE6BF450BF6F58DFF450B9D79D
:10146000B000B0C09BF0B1C09CF0B2C09DF0B3C062
:101470009EF00101076B0001B351B011B111B2111F
:10148000D8B4B3D00001B45186D7B000B0C09BF03F
:10149000B1C09CF0B2C09DF0B3C09EF00101076BDB
:1014A0000001B351B011B111B211D8B49ED00001F6
:1014B000B4518FD7B000B0C09BF0B1C09CF0B2C0A7
:1014C0009DF0B3C09EF00101076B0001B351B01154
:1014D000B111B211D8B489D00001B45192D7E16EE4
:1014E0000A0E0001BB6FBC6BBD6BBE6BE150BF6FE2
:1014F0000DDF010E0001BB6FBC6BBD6BBE6BE1501D
:10150000BF6F04D7B0000001E8CF9BF09C6B9D6BD0
:101510009E6B0101076B0001B051E1D7BA000001D9
:10152000E8CF9BF09C6B9D6B9E6B0101076B640E7B
:101530000001BB6FBC6BBD6BBE6BBA51BF6FE6DE0B
:101540000001BA51CCD7C4000001C551ACDE000186
:10155000C451A9D6C0000001C251A5DEC0C0C4F06C
:10156000C1C0C5F0F1D7B0000001B3519CDEB0C0DE
:10157000C0F0B1C0C1F0B2C0C2F0B3C0C3F0EBD78D
:10158000B4000001B7AF0ED02D0E7EDE046A056AEE
:10159000800E066EBF0E076EB40EE96E000EEA6E88
:1015A0003CEC30F0B4C000F0B5C001F0B6C002F0C1
:1015B000B7C003F00AEC2FF000500001B96FB95129
:1015C000D8A403D0300E60DE04D00001BA6BB9514C
:1015D000A6DF2E0E59DEB40EE96E000EEA6EEE5056
:1015E000EE10EE10EE10D8A402D0300E4DD6D96A0F
:1015F0000001B851D95CD8B01200B9C000F0C6ECF7
:101600002FF000C004F001C005F002C006F003C0D6
:1016100007F0B40EE96E000EEA6E06EC30F0046AD4
:10162000056A200E066E410E076EB40EE96E000EBE
:10163000EA6E3CEC30F0B40EE96E000EEA6EEE504D
:10164000EE10EE10EE10D8B41200B4C000F0B5C029
:1016500001F0B6C002F0B7C003F00AEC2FF0005062
:101660000001B96FB951300F0FDED92AC1D73B0E37
:101670000BDE0D0E09DE95EF14F03DBA3EA423D02B
:1016800053C000F054C001F055C002F056C003F042
:10169000046A056A066A0350076E075004100510B5
:1016A0000610D8A410D000EE63F000015351EE18DC
:1016B00008E15451EE1805E15551EE1802E156517A
:1016C000EE18D8A4120005C1E8FF020AD8A423D05E
:1016D000F36A07D0F3502E0FE96EEA6AEF50E3DDAC
:1016E000F32A1450D8A402D0070E01D00E0E006EBB
:1016F000016AF3CF02F0036A0350800A046E0150BE
:10170000800A045C02E10050025CD8A0E3D70D0E11
:10171000BBDD95EF14F005C1E8FF030AD8A422D081
:101720002A0EB2DDF36A07D0F3502E0FE96EEA6A93
:10173000EF50B9DDF32A1450D8A402D0070E01D01F
:101740000E0E006E016AF3CF02F0036A0350800AA6
:10175000046E0150800A045C02E10050025CD8A0D3
:10176000E3D785D705C1E8FF040AD8A42FD0400EDF
:101770008BDD97C0B0F098C0B1F099C0B2F09AC0BC
:10178000B3F0F2DECF508FDD18508DDDF36A07D055
:10179000F3502E0FE96EEA6AEF5085DDF32A1450FC
:1017A000D8A402D0070E01D00E0E006E016AF3CF4E
:1017B00002F0036A0350800A046E0150800A045C40
:1017C00002E10050025CD8A0E3D751D705C1E8FF81
:1017D000080AD8A420D0FF0E57DDD96AD9502E0FA1
:1017E000E96EEA6AEF5050DDD92A060ED964F6D7C1
:1017F000070ED96E1450D8B407D0D9502E0FE96E09
:10180000EA6AEF5041DD02D0000E3EDDD92A0D0E0E
:10181000D964F0D7120005C1E8FF090AD8A424D082
:101820002F0E32DDF36A07D0F3502E0FE96EEA6A0D
:10183000EF5039DDF32A1450D8A402D0070E01D09E
:101840000E0E006E016AF3CF02F0036A0350800AA5
:10185000046E0150800A045C02E10050025CD8A0D2
:10186000E3D705DF3E803D9E05C100F00004D8A40B
:1018700008D001C1E8FF020AD8A403D0010EE8CFC6
:1018800001F101010153D8A402D02D0EFDDC01C1EC
:1018900000F00004D8A402D02B0EF6DC01C1E8FF52
:1018A000020AD8A402D02A0EEFDC3EB020D0F36AA0
:1018B00007D0F3502E0FE96EEA6AEF50F4DCF32AFA
:1018C0001450D8A402D0070E01D00E0E006E016A8B
:1018D000F3CF02F0036A0350800A046E0150800ABD
:1018E000045C02E10050025CD8B0C1D6E2D73DAE44
:1018F0001FD0F36A07D0F3502E0FE96EEA6AEF505B
:10190000D2DCF32A1450D8A402D0070E01D00E0E58
:10191000006E016AF3CF02F0036A0350800A046E7E
:101920000150800A045C02E10050025CD8A0E3D7B9
:101930002C0EAADC45C000F046C001F0000E01BE2E
:10194000FF0E026E036E00C0B0F001C0B1F002C025
:10195000B2F003C0B3F00001B46B83DD2C0E94DC55
:10196000010E0001B06F03C1E8FFCDDD2C0E8CDC51
:101970003EA409D063C0C0F064C0C1F065C0C2F02D
:1019800066C0C3F0E8DD2C0E7FDC01010853D8B43B
:1019900006D00001080EB06F010EB16F8CDC2C0E6A
:1019A00073DC01010853D8B403D004C1E8FF6CDC38
:1019B0002C0E6ADC3EAA06D03DB202D0300E01D019
:1019C000310E62DC2C0E60DC3DAC66D03EAA1CD031
:1019D0006BC0B0F06CC0B1F06DC0B2F06EC0B3F0CF
:1019E00000EEB4F06FC0EEFF70C0EEFF71C0EEFF0E
:1019F00072C0EEFF000E3DB4010E0001B86F000E84
:101A00003DB2010E81EC05F03DA824D03EAA0DD0D8
:101A100009EC07F000C0B0F001C0B1F002C0B2F0B4
:101A200003C0B3F00001B46B46DD2C0E2DDC3EAAE2
:101A30000ED0F6EC07F000C0B4F001C0B5F002C063
:101A4000B6F003C0B7F0040E0001B86F9ADD2C0E9B
:101A50001BDC42D03EAA0CD073C0B4F074C0B5F009
:101A600075C0B6F076C0B7F0060E0001B86F89DD1C
:101A70002C0E0ADC3EAA0CD07BC0B4F07CC0B5F0C2
:101A80007DC0B6F07EC0B7F0060E0001B86F79DDFC
:101A90002C0E44EC09F020D03EAA0BD06BC0B0F065
:101AA0006CC0B1F06DC0B2F06EC0B3F00001B46BA9
:101AB000EDDC2C0E44EC09F03EAA0BD06FC0B0F068
:101AC00070C0B1F071C0B2F072C0B3F00001B46B7D
:101AD000DDDC2C0E44EC09F03EA620D03DA403D062
:101AE000400E44EC09F06AC0E8FFE8AE0CD02D0EC1
:101AF00044EC09F0FF0E046805680668076800EE0C
:101B000067F028EC30F067C0B0F068C0B1F069C091
:101B1000B2F06AC0B3F00001B46BB8DC2C0E44EC38
:101B200009F03EAE05D047C0C4F048C0C5F00CDD9A
:101B30002C0E44EC09F03FA428D04EC0E8FFE8AEDC
:101B400010D02D0E44EC09F0FF0E026803684DC062
:101B500000F04EC001F0DCEC2FF004C04DF005C0E9
:101B60004EF04DC000F04EC001F0000E01BEFF0E61
:101B7000026E036E00C0B0F001C0B1F002C0B2F05E
:101B800003C0B3F00001B46B6CDC2C0E44EC09F024
:101B90003EAC28D044C0E8FFE8AE10D02D0E44EC97
:101BA00009F0FF0E0268036843C000F044C001F072
:101BB000DCEC2FF004C043F005C044F043C000F05B
:101BC00044C001F0000E01BEFF0E026E036E00C0A5
:101BD000B0F001C0B1F002C0B2F003C0B3F0000138
:101BE000B46B3FDC2C0E44EC09F03FA228D04AC075
:101BF000E8FFE8AE10D02D0E44EC09F0FF0E0268AD
:101C0000036849C000F04AC001F0DCEC2FF004C0CA
:101C100049F005C04AF049C000F04AC001F0000E8A
:101C200001BEFF0E026E036E00C0B0F001C0B1F045
:101C300002C0B2F003C0B3F00001B46B12DC2C0E92
:101C400044EC09F03FA00CD093C0B4F094C0B5F0C0
:101C500095C0B6F096C0B7F0050E0001B86F91DCE4
:101C60002C0E44EC09F03EA802D5000E3EB8010E41
:101C70000001B06FB16BB26BB36BB46B31EC0AF0B7
:101C8000F6D4D96E2F0ED96406D03A0ED96003D09F
:101C9000D950D00F1200400ED96406D0470ED9603B
:101CA00003D0D950C90F1200600ED964000C670E22
:101CB000D960000CD950A90F1200200E0001B06F9E
:101CC0004C0E44EC09F0610E44EC09F0740E44EC47
:101CD00009F03A0E44EC09F00001B16B0001B20EBC
:101CE000B76F000EB86F36EC09F0D8A0F7D7000137
:101CF000B25144EC09F00001B251C3DF0001B36FEF
:101D0000B46BB56BB66B0001B20EB76F000EB86F57
:101D100036EC09F0D8A0F7D70001B25144EC09F035
:101D2000040EB3C000F0B4C001F0B5C002F0B6C0FC
:101D300003F012EC30F00001B251A3DF00100001FB
:101D4000B36F0150B46F0250B56F0350B66FFBEC28
:101D500001F00001B051A96EB02BB351A86E3F0E37
:101D6000A616D890F2BED880F29EA684550EA76E15
:101D7000AA0EA76EA682A198A694D8B0F28EB12B17
:101D8000030EB165ABD70D0E44EC09F00A0E44EC1E
:101D900009F0240E0001B06F4C0E44EC09F06F0EF8
:101DA00044EC09F06E0E44EC09F03A0E44EC09F0F4
:101DB0000001B16B0001B20EB76F000EB86F36ECC8
:101DC00009F0D8A0F7D70001B25144EC09F00001A6
:101DD000B25157DF0001B36FB46BB56BB66B000146
:101DE000B20EB76F000EB86F36EC09F0D8A0F7D777
:101DF0000001B25144EC09F0040EB3C000F0B4C0CD
:101E000001F0B5C002F0B6C003F012EC30F00001F2
:101E1000B25137DF00100001B36F0150B46F0250B0
:101E2000B56F0350B66FFBEC01F00001B051A96E25
:101E3000B02BB351A86E3F0EA616D890F2BED88034
:101E4000F29EA684550EA76EAA0EA76EA682A19832
:101E5000A694D8B0F28EB12B030EB165ABD70D0EA0
:101E600044EC09F00A0E44EC09F040EF04F07C0E5B
:101E700044EC09F0200E66EC03F000C0B0F001C0A5
:101E8000B1F002C0B2F003C0B3F0B0C0B4F0B1C062
:101E9000B5F0B2C0B6F0B3C0B7F0060EB86FC1EC83
:101EA0000AF02C0E44EC09F0240E66EC03F000C09E
:101EB000B0F001C0B1F002C0B2F003C0B3F0B0C0E6
:101EC000B4F0B1C0B5F0B2C0B6F0B3C0B7F0060E12
:101ED000B86FC1EC0AF037EF0BF00001536B546B95
:101EE000556B566B0001B66B00EE53F0080ED890A0
:101EF000EE36EE36EE36ED36ED52ED52E82EF7D7F1
:101F0000FBEC01F00001B651280FA96E3F0EA6169A
:101F1000A680A85000EE53F0EE12000EEE12EE1264
:101F2000ED12ED52ED52B62B030EB665DDD7120061
:101F3000FBEC01F0280EA96EA8683F0EA616D890FB
:101F4000F2BED880F29EA684550EA76EAA0EA76E8A
:101F5000A682A198A694D8B0F28EBFD73E0E44ECCC
:101F600009F053C000F054C001F055C002F056C053
:101F700003F0046A056A066A0350076E07500410EE
:101F800005100610D8A437EF0BF053C0C0F054C0B2
:101F9000C1F055C0C2F056C0C3F0ABEC0AF037EF49
:101FA0000BF0430E44EC09F06F0E44EC09F0640EA4
:101FB00044EC09F0650E44EC09F03A0E44EC09F0EB
:101FC000FBEC01F0280EA96EA86A3F0EA616D89069
:101FD000F2BED880F29EA684550EA76EAA0EA76EFA
:101FE000A682A198A694D8B0F28E010E0001B06F1F
:101FF0000001B10EB76F000EB86F36EC09F0D8A033
:10200000F7D70001B15144EC09F00001B15139DEBC
:102010000001B26FB36BB46BB56B0001B10EB76F5B
:10202000000EB86F36EC09F0D8A0F7D70001B15117
:1020300044EC09F0040EB2C000F0B3C001F0B4C02B
:1020400002F0B5C003F012EC30F00001B15119DE1E
:1020500000100001B26F0150B36F0250B46F035013
:10206000B56FFBEC01F00001B051280FA96EB25121
:10207000A86E3F0EA616D890F2BED880F29EA68417
:10208000550EA76EAA0EA76EA682A198A694D8B0E8
:10209000F28EB02B030EB065ABD70D0E44EC09F0F9
:1020A0000A0E44EC09F019D73D0E44EC09F000018A
:1020B000B06BB16B180EB26FB36B6CEC09F037EF0D
:1020C0000BF0240E44EC09F0430E44EC09F0520EE0
:1020D00044EC09F0430E44EC09F03A0E44EC09F0EC
:1020E00081B602D0300E01D0310E44EC09F02C0E36
:1020F00044EC09F0310E44EC09F0310E44EC09F0E7
:10210000320E44EC09F03A0E44EC09F081B402D0EE
:10211000300E01D0310E44EC09F02C0E44EC09F0E5
:10212000450E44EC09F0580E44EC09F0540E44EC12
:1021300009F03A0E44EC09F03EB002D0300E01D066
:10214000310E44EC09F02C0E44EC09F0520E44EC34
:1021500009F0410E44EC09F0570E44EC09F03A0E38
:1021600044EC09F03DBE02D0300E01D0310E44ECFB
:1021700009F02C0E44EC09F0500E44EC09F04F0E1F
:1021800044EC09F0530E44EC09F03A0E44EC09F02B
:102190003DBC02D0300E01D0310E44EC09F02C0EC3
:1021A00044EC09F0440E44EC09F0530E44EC09F001
:1021B000540E44EC09F03A0E44EC09F03DB802D05C
:1021C000300E01D0310E44EC09F02C0E44EC09F035
:1021D000460E44EC09F04C0E44EC09F0540E44EC6D
:1021E00009F03A0E44EC09F03DBA02D0300E01D0AD
:1021F000310E44EC09F02C0E44EC09F0410E44EC95
:1022000009F04C0E44EC09F0520E44EC09F03A0E81
:1022100044EC09F03DB602D0300E01D0310E44EC52
:1022200009F02C0E44EC09F04D0E44EC09F0440E7C
:1022300044EC09F0450E44EC09F03A0E44EC09F088
:1022400005C1E8FF300F44EC09F02C0E44EC09F016
:10225000410E44EC09F0430E44EC09F0520E44ECFC
:1022600009F03A0E44EC09F000C1E8FF300F44ECED
:1022700009F037EF0BF0230E44EC09F022C0B0F068
:1022800023C0B1F024C0B2F025C0B3F0010E0001AC
:10229000B46F5BEC0AF02C0E44EC09F02AC0B0F0ED
:1022A0002BC0B1F02CC0B2F02DC0B3F0010E000174
:1022B000B46F5BEC0AF02C0E44EC09F01AC0B0F0DD
:1022C0001BC0B1F01CC0B2F01DC0B3F0010E000184
:1022D000B46F5BEC0AF02C0E44EC09F026C0B0F0B1
:1022E00027C0B1F028C0B2F029C0B3F0010E000140
:1022F000B46F5BEC0AF02C0E44EC09F01EC0B0F099
:102300001FC0B1F020C0B2F021C0B3F0010E000137
:10231000B46F5BEC0AF02C0E44EC09F04BC0C4F037
:102320004CC0C5F0A4EC0AF037EF0BF081A67CD0CE
:10233000026A5E0E44EC09F0010E0001BA6F025011
:102340008FEC0AF02C0E44EC09F002500B0D110E2C
:10235000F324E96E010EF420EA6EEECFC0F0EECF6A
:10236000C1F0EECFC2F0EECFC3F0ABEC0AF02C0E12
:1023700044EC09F002500B0D170EF324E96E010E28
:10238000F420EA6EEECFF6FFEDCFF7FFF628D8B4D3
:10239000F728D8B406D0F6CFC4F0F7CFC5F0A4EC38
:1023A0000AF02C0E44EC09F0010E0001B06F02504F
:1023B0000B0D1B0EF324E96E010EF420EA6EEF50B4
:1023C00083EC0AF02C0E44EC09F002500B0D190EB0
:1023D000F324E96E010EF420EA6EEECF00F0EDCFAB
:1023E00001F000500001B06F0150B16FB26BB36BE0
:1023F000010EB46F46EC0AF02C0E44EC09F00250CA
:102400000B0D150EF324E96E010EF420EA6EEECFEB
:10241000C4F0EDCFC5F0A4EC0AF037EC0BF0022AC3
:10242000410E026486D712005E0E44EC09F037EFCD
:102430000BF03C0E44EC09F063C0C0F064C0C1F086
:1024400065C0C2F066C0C3F0ABEC0AF037EF0BF02A
:10245000B800E96E210E44EC09F063C0C0F064C01E
:10246000C1F065C0C2F066C0C3F0ABEC0AF02C0E40
:1024700044EC09F0E95044EC09F02C0E44EC09F06E
:102480000001B85144EC09F037EF0BF0D96AD9508C
:102490000B0D150EF324E96E010EF420EA6EEE6AC0
:1024A000ED6AD9500B0D110EF324E96E010EF420E4
:1024B000EA6EEE6AEE6AEE6AED6AD9500B0D170EFF
:1024C000F324E96E010EF420EA6EEE68ED68D9504F
:1024D0000B0D1B0EF324E96E010EF420EA6EEF6A79
:1024E000D9500B0D190EF324E96E010EF420EA6E9B
:1024F000EE6AED6AD92A410ED964C9D712000001EB
:10250000C06FD96A00EE63F0D9500B0D110EF324A1
:10251000E16E010EF420E26EE650EE1808E1E6509E
:10252000EE1805E1E650EE1802E1E650EE18D8A4E8
:102530001ED0C0C000F0016A026A036AD9500B0DB8
:10254000110EF324E96E010EF420EA6EEE52EE5203
:10255000EE520350ED5C08E10250ED5C05E10150E4
:10256000ED5C02E10050EF5CD8B0010C000CD92A00
:10257000410ED964C7D7000C016E0268D96A0228DF
:10258000D8A40DD0D9500B0D1B0EF324E96E010E0B
:10259000F420EA6EEF50D8A402D0D950026E00EEBB
:1025A00063F0D9500B0D110EF324E16E010EF420EF
:1025B000E26EE650EE1808E1E650EE1805E1E6504E
:1025C000EE1802E1E650EE18D8A438D0D9500B0D21
:1025D0001B0EF324E96E010EF420EA6EEF50006E3C
:1025E0000150005CD8B00AD0D9500B0D1B0EF3245B
:1025F000E96E010EF420EA6E01C0EFFFD60E4BC06B
:1026000000F04CC001F00026000E0122D9500B0D45
:10261000150EF324E96E010EF420EA6E00C0EEFF01
:1026200001C0EDFFD9500B0D190EF324E96E010E18
:10263000F420EA6EEE2A000EED22010CD92A410E9A
:10264000D9649DD70228D8B4000C0104D8B4000C7A
:1026500002500B0D110EF324E96E010EF420EA6E08
:1026600063C0EEFF64C0EEFF65C0EEFF66C0EEFF24
:1026700002500B0D170EF324E96E010EF420EA6EE2
:10268000EE68ED6802500B0D1B0EF324E96E010E8F
:10269000F420EA6E01C0EFFFD60E4BC000F04CC034
:1026A00001F00026000E012202500B0D150EF3243E
:1026B000E96E010EF420EA6E00C0EEFF01C0EDFFEE
:1026C000D9500B0D190EF324E96E010EF420EA6EB9
:1026D000010EEE6EED6A000CD96A00EE63F0D9507F
:1026E0000B0D110EF324E16E010EF420E26EE650A4
:1026F000EE1808E1E650EE1805E1E650EE1802E1AA
:10270000E650EE18D8A40DD0D9500B0D170EF324B7
:10271000E96E010EF420EA6E47C0EEFF48C0EDFFFF
:10272000010CD92A410ED964D8D7000C490E44ECCB
:1027300009F0320E44EC09F0430E44EC09F03A0E75
:1027400044EC09F00001B20EB76F000EB86F36EC22
:1027500009F0D8A0F7D70001B25144EC09F000010C
:10276000B25141EC0EF00001B16F0001B20EB76F33
:10277000000EB86F36EC09F0D8A0F7D70001B251BF
:1027800044EC09F00001B25141EC0EF0016EB1C011
:1027900000F0003AF00E0016015000100001B16F79
:1027A000100EB16501D01200FBEC01F06E0EA96EA7
:1027B0000001B151A86E3F0EA616D890F2BED88087
:1027C000F29EA684550EA76EAA0EA76EA682A198A9
:1027D000A694D8B0F28EB151D8B45AD0B06B54D0C0
:1027E0000001B20EB76F000EB86F36EC09F0D8A03A
:1027F000F7D70001B25144EC09F00001B25141ECAD
:102800000EF00001B36FB46BB56BB66B0001B20E86
:10281000B76F000EB86F36EC09F0D8A0F7D70001FB
:10282000B25144EC09F0040EB3C000F0B4C001F0A2
:10283000B5C002F0B6C003F012EC30F00001B251A6
:1028400041EC0EF000100001B36F0150B46F025064
:10285000B56F0350B66FFBEC01F00001B0516F0F84
:10286000A96EB351A86E3F0EA616D890F2BED880BE
:10287000F29EA684550EA76EAA0EA76EA682A198F8
:10288000A694D8B0F28EB02B0001B051B161A8D798
:102890000D0E44EC09F049D0490E44EC09F0320E1B
:1028A00044EC09F0430E44EC09F03A0E44EC09F014
:1028B000FBEC01F06E0EA96E3F0EA616A680A85086
:1028C0000001B06FB051D8A407D04E0E44EC09F00F
:1028D0004F0E44EC09F026D0400E44EC09F0FBEC1E
:1028E00001F06F0EA96E3F0EA616A680A85053ECFD
:1028F00009F07C0E44EC09F0010E0001B16F0ED01E
:10290000FBEC01F00001B1516F0FA96E3F0EA6164E
:10291000A680A85053EC09F00001B12B0001B15181
:10292000B061EED70D0E44EC09F00A0E44EF09F049
:10293000B0000001B26FFBEC01F00001B151A96ED3
:102940003F0EA616A680A850B16FB151D8A402D0F0
:10295000D8801200100E0001B16502D0D88012009C
:102960003D0E44EC09F0490E44EC09F0320E44EC03
:1029700009F0430E44EC09F0200E44EC09F09E9659
:10298000C580F368F46803D0F306D8A0F406F450C9
:10299000C5A004D0F310D8A4F7D7F450F310D8B4DE
:1029A00079D0FBEC01F00001B251A96E3F0EA616E2
:1029B000A680A850E96E400E44EC09F0E95053ECB3
:1029C00009F09E96E950C96EF368F46803D0F306E7
:1029D000D8A0F406F450C7A404D0F310D8A4F7D7B5
:1029E000F450F310D8B456D0F368F46803D0F3066B
:1029F000D8A0F406F450C5AC04D0F310D8A4F7D78F
:102A0000F450F310D8B446D07C0E44EC09F0000129
:102A1000B151D8B434D09E96FBEC01F00001B05116
:102A2000A96EB02B3F0EA616A680A850E96EE950FD
:102A300053EC09F0E950C96EF368F46803D0F3066B
:102A4000D8A0F406F450C7A404D0F310D8A4F7D744
:102A5000F450F310D8B41ED0F368F46803D0F30632
:102A6000D8A0F406F450C5AC04D0F310D8A4F7D71E
:102A7000F450F310D8B40ED00001B107C8D7D96A0A
:102A80003A0E44EC09F04F0E44EC09F04B0E44ECC6
:102A900009F00BD0010ED96E3A0E44EC09F04B0E42
:102AA00044EC09F04F0E44EC09F00D0E44EC09F033
:102AB0000A0E44EC09F0C584F368F46803D0F30609
:102AC000D8A0F406C5B4FBD7F450F310D8A4F7D7B8
:102AD0009E96D9CF00F000301200B800F36AF46A75
:102AE0000001BC6BBD6BB9B7F384B9B5BC8BB9B38E
:102AF000F382B9B1BC89B8BFF380B8BDBC87B8BB9D
:102B0000BC85B8B7BC83B8B5BC8FB8B3BC81B8B10D
:102B1000BC8DBCC000F0BDC001F0040E026ED890A8
:102B200001320032022EFBD700010050BC1B0150C5
:102B3000BD1BBCC000F0BDC001F0D8900132003216
:102B4000D890013200320050BC1B0150BD1BD89000
:102B5000BD31016EBC31006E0050BC1B0150BD1B6D
:102B6000FF0EF324026EFF0EF420036EBCA104D00E
:102B7000060E0226000E0322D8900234006E0334A3
:102B8000016E0050000FF66E0150F76E040EF72232
:102B90000900F5CFBAF00900F5CFBBF0050E026EC3
:102BA000036ABCC000F0BDC001F0DCEC2FF00001F6
:102BB000BA510426BB510522FF0E0424BC6FFF0E40
:102BC0000520BD6FBCC000F0BDC001F01200C00008
:102BD000800E006E040E016EFA0E026E0368D96A52
:102BE0000001C3AF08D00050C01B0150C11B0250F0
:102BF000C21B0350C31B0001D890C037C137C23776
:102C0000C337D92A1F0ED964EBD7C0C000F0C1C0AA
:102C100001F0C2C002F0C3C003F01200C000000106
:102C2000800ECC6F040ECD6FFA0ECE6FCF69D96ACD
:102C30000001C3AF08D0CC51C01BCD51C11BCE5138
:102C4000C21BCF51C31B1F0EC4C000F0C5C001F092
:102C5000C6C002F0C7C003F01DEC30F0010E001436
:102C6000046E056A066A076A0001D890C035006ED6
:102C7000C135016EC235026EC335036E00500424A7
:102C8000C06F01500520C16F02500620C26F035073
:102C90000720C36F1F0EC8C000F0C9C001F0CAC032
:102CA00002F0CBC003F01DEC30F0010E0014046EF6
:102CB000056A066A076AD890C435006EC535016E8C
:102CC000C635026EC735036E00500424C46F015030
:102CD0000520C56F02500620C66F03500720C76F3E
:102CE000D890C837C937CA37CB37D92A570ED964D5
:102CF0009FD7C0C000F0C1C001F0C2C002F0C3C085
:102D000003F012000101016BB80EE16E000EE26EDD
:102D100031C0E6FF30C0E6FF2FC0E6FF2EC0E6FF61
:102D2000B6D0BC0EE16E000EE26EE1CFE9FFE2CF5D
:102D3000EAFFE14AE22AEF6A34C0E6FF33C0E6FF69
:102D400032C0E6FFB8C0C0F0B9C0C1F0BAC0C2F02E
:102D5000BBC0C3F03DDF00010050BC1B0150BD1BD8
:102D60000250BE1B0350BF1BBDC0BCF0BEC0BDF0B7
:102D7000BFC0BEF0BF6B070E006ED890BF33BE332E
:102D8000BD33BC33002EF9D7BF51BC11BD11BE11EC
:102D9000010ED8A405D0E8CF01F1020EBCEF12F06D
:102DA0001A26000E1B221C221D221200B00EE16EFC
:102DB000000EE26E35C0E6FF34C0E6FF33C0E6FF2A
:102DC00032C0E6FFB40EE16E000EE26EE1CFE9FF25
:102DD000E2CFEAFFE14AE22AEF6A38C0E6FF37C0F5
:102DE000E6FF36C0E6FFBC0EE16E000EE26EE1CFFC
:102DF000E9FFE2CFEAFFE14AE22AEF6A3BC0E6FFE1
:102E00003AC0E6FF39C0E6FFB8C0C0F0B9C0C1F0B3
:102E1000BAC0C2F0BBC0C3F0B0C0C4F0B1C0C5F00E
:102E2000B2C0C6F0B3C0C7F0B4C0C8F0B5C0C9F0F6
:102E3000B6C0CAF0B7C0CBF0F2DE00010050BC1B38
:102E40000150BD1B0250BE1B0350BF1BBF51BC1124
:102E5000BD11BE11010ED8A405D0E8CF01F1030EBB
:102E6000BCEF12F01A26000E1B221C221D2212009B
:102E7000010E7FEC12F00009D8B405D0010EE8CFA6
:102E800001F1BCEF12F0020EE8CF01F1120003C114
:102E9000E8FF0B0A01E145D71A0A88E0030A86E039
:102EA000010AE6E0E5D73E94BC0EE16E000EE26E4C
:102EB00031C0E6FF30C0E6FF2FC0E6FF2EC0E6FFC0
:102EC000C0D01AD10001BCC063F0BDC064F0BEC068
:102ED00065F0000EE8CF66F02BD01AD03238E84605
:102EE0001F0BD96E000ED96404D0050ED96001D035
:102EF0000FD0D950130AD8A403D033BEFDD008D0C8
:102F0000040ED96407D0090ED96004D034B6F4D0C9
:102F10003E84F2D0080ED964EFD0170ED960ECD001
:102F200032B0EAD0F5D732BEE7D0F2D7E5D0F0D74D
:102F300002C1E8FF000AD1E0010ACFE0030ACEE0B7
:102F4000010AF1E0070AF2E0010AF1E0030AEFE00A
:102F5000D3D00001BCC063F0BDC064F0BEC065F05A
:102F6000000EBF15E8CF66F0D3D7B00EE16E000EAD
:102F7000E26E35C0E6FF34C0E6FF33C0E6FF32C084
:102F8000E6FFB40EE16E000EE26EE1CFE9FFE2CFA4
:102F9000EAFFE14AE22AEF6A38C0E6FF37C0E6FFFF
:102FA00036C0E6FFB80EE16E000EE26EE1CFE9FF3B
:102FB000E2CFEAFFE14AE22AEF6A3BC0E6FF3AC00D
:102FC000E6FF39C0E6FFBCC0C0F0BDC0C1F0BEC066
:102FD000C2F0BFC0C3F0B0C0C4F0B1C0C5F0B2C051
:102FE000C6F0B3C0C7F0B4C0C8F0B5C0C9F0B6C031
:102FF000CAF0B7C0CBF013DE00C063F001C064F0CC
:1030000002C065F003C066F000EE63F00001B85145
:10301000EE1AB951EE1ABA51EE1ABB51ED1AED5231
:10302000ED5200EE63F0080EEC52EC52EC52D890E8
:10303000ED32ED32ED32EF32E82EF6D769D73E842D
:103040001FD003C1E8FF000AFAE0040AF8E0010A11
:10305000F6E00E0A01E17DD71B0A87E0010A01E1D3
:1030600078D7030A01E12ED7010A01E12AD7070A1E
:1030700001E17BD7010A01E178D70D0A01E175D79B
:10308000B80EE16E000EE26EE1CFE9FFE2CFEAFF9B
:10309000E14AE22AEF6A34C0E6FF33C0E6FF32C0FD
:1030A000E6FFBCC0C0F0BDC0C1F0BEC0C2F0BFC032
:1030B000C3F08EDD00C063F001C064F002C065F0B3
:1030C00003C066F000EE63F00001B851EE1AB9518A
:1030D000EE1ABA51EE1ABB51ED1AED52ED5200EE56
:1030E00063F0080EEC52EC52EC52D890ED32ED3217
:1030F000ED32EF32E82EF6D73EB43DA6120000EED8
:1031000063F000015351EE1808E15451EE1805E147
:103110005551EE1802E15651EE18D8A412008098CD
:1031200019EC12F080881200D96E000ED96406D016
:103130001B0ED96003D0D950400F12002F0ED96456
:10314000200C3A0ED960200CD95012000101086BF6
:103150000101046B3D943F943E9C3F923F903E980A
:103160003E9A3E963E9E13EF1DF002D00ED0120006
:1031700002C1E8FF000AFAE0010AF8E0030AF6E0FB
:10318000010AF5E0050AF2E012003238E8461F0BAA
:10319000D96E34D3440E05D0430E03D0420E01D075
:1031A000410EE8CF04F1F46AF36A036A6DD0F32AA2
:1031B000F30411EE08F0E126000EE222F450330F82
:1031C000E96EEA6AEF50006ED8900032D890003075
:1031D0003F0BAADFE76EF32AF30411EE08F0E126B5
:1031E000000EE222F450340FE96EEA6AEF50016EED
:1031F000013A0F0E01160116F450330FE96EEA6A18
:10320000EF50006E003AF00E0016300E001601501E
:1032100000108ADFE76EF32AF30411EE08F0E126CE
:10322000000EE222F450350FE96EEA6AEF50016EAB
:10323000060E006ED8900132002EFCD7030E011648
:10324000F450340FE96EEA6AEF50006E020E026E1F
:10325000D8900036022EFCD73C0E0016015000100C
:1032600063DFE76EF32AF30411EE08F0E126000EA7
:10327000E222F450350FE96EEA6AEF503F0B54DF5B
:10328000E76E030EF426032A010E036490D7F32A97
:10329000F30401EE08F0E926000EEA22EF6A1200BC
:1032A0003D843E867DD033500001B26FB36BB2C017
:1032B00000F0B3C001F0003A013AF00E01160050E0
:1032C0000F0B0112F00E001634380F0B0010B26F06
:1032D0000150B36FB351B211D8B45FD0B2A92DD0A1
:1032E0000F0EB2C000F0B3C001F00016016AD89012
:1032F000B331036EB231026EF00BF66E0350F76E0F
:103300000050F610B26F0150F710B36F190E026E35
:10331000036AB2C000F0B3C001F0DCEC2FF0180E6D
:103320000424E8CF67F0FC0E0520E8CF68F0000E1B
:10333000E8CF69F0E8CF6AF02FD0B2C0B8F0B3C0E0
:10334000B9F06EEC15F000C0B0F001C0B1F00001B2
:10335000B151B011D8B421D0640E046E056A066A6A
:10336000076AB0C000F0B1C001F0000E01BEFF0E50
:10337000026E036E6BEC2EF000C067F001C068F0C7
:1033800002C069F003C06AF00001B40E6727FB0EAB
:103390006823FF0E69236A233E86D950D8B41200F1
:1033A00034C000F0020E016ED8900032012EFCD71E
:1033B00000303D92D8B03D8234C000F0030E0016BC
:1033C000000100C06BF06C6B6D6B6E6B080E6BC018
:1033D00000F06CC001F06DC002F06EC003F012ECA2
:1033E00030F035C004F0056A066A076A0450001020
:1033F000E8CF6BF005500110E8CF6CF006500210DA
:10340000E8CF6DF007500310E8CF6EF0070E6BC0E9
:1034100000F06CC001F06DC002F06EC003F012EC61
:1034200030F000C0B4F001C0B5F002C0B6F003C087
:10343000B7F036C000F0010E016ED8900032012EB8
:10344000FCD700C004F0056A066A076A0001045050
:10345000B411E8CF6BF00550B511E8CF6CF0065011
:10346000B611E8CF6DF00750B711E8CF6EF036C057
:1034700000F0010E0016000100C06FF0706B716B60
:10348000726B080E6FC000F070C001F071C002F0E6
:1034900072C003F012EC30F037C004F0056A066A1F
:1034A000076A04500010E8CF6FF005500110E8CF14
:1034B00070F006500210E8CF71F007500310E8CF0B
:1034C00072F0080E6FC000F070C001F071C002F021
:1034D00072C003F012EC30F038C004F0056A066ADE
:1034E000076A04500010E8CF6FF005500110E8CFD4
:1034F00070F006500210E8CF71F007500310E8CFCB
:1035000072F03E8A12000001436B446B496B4A6BB8
:10351000936B946B956B966B416B426B040ED96EFB
:10352000F6D0010ED96E33C000F0030E0016000174
:1035300000C043F0446B34C002F0036A4351016E93
:10354000006A02500010E8CF43F003500110E8CFAA
:1035500044F043514411D8B421D0D9CF02F0036ACA
:1035600043C000F044C001F0FF0E00060120016ED0
:10357000DCEC2FF004C043F005C044F033A40DD0C0
:10358000FF0E0268036843C000F044C001F0DCECA9
:103590002FF004C043F005C044F03E8C35C000F06D
:1035A0007F0E0016000100C049F04A6B36C000F0E3
:1035B000050E016ED8900032012EFCD700C002F03B
:1035C000036A49C000F04AC001F0D89000360136C5
:1035D000D89000360136D8900036013602500010DF
:1035E000E8CF49F003500110E8CF4AF049514A11A1
:1035F000D8B4A3D0D9CF02F0036A49C000F04AC0C2
:1036000001F0FF0E00060120016EDCEC2FF004C07B
:1036100049F005C04AF035AE0DD0FF0E02680368D0
:1036200049C000F04AC001F0DCEC2FF004C049F0C2
:1036300005C04AF03F8281D0010ED96E3F903FA075
:1036400027D03350030BF66EF76AF650F76E34C08E
:10365000E8FFF66EF6CF00F0F7CF01F0F3EC2FF0B5
:10366000046A056AB40E066E430E076ECEEC2CF0AB
:10367000046A056A800E066E440E076E23EC27F07E
:1036800000C093F001C094F002C095F003C096F022
:1036900035C000F07F0E0016000100C041F0426B03
:1036A00036C000F0050E016ED8900032012EFCD716
:1036B00000C002F0036A41C000F042C001F0D8909F
:1036C00000360136D89000360136D89000360136E3
:1036D00002500010E8CF41F003500110E8CF42F053
:1036E00041514211D8B429D0D9CF02F0036A41C068
:1036F00000F042C001F0FF0E00060120016EDCEC7C
:103700002FF004C041F005C042F03E8816D032C010
:1037100000F0070E001600C002F0036A0CD0025041
:10372000010A01E1FED6030A01E1FDD6010A84E0A7
:10373000070A84E002D00350F2E036C000F0070E22
:103740000016000100C04DF04E6B37C000F0020EB5
:10375000016ED8900032012EFCD700C002F0036A3F
:103760004DC000F04EC001F0060ED8900036013674
:10377000E82EFBD702500010E8CF4DF003500110A7
:10378000E8CF4EF04D514E11D8B412004DC000F0AC
:103790004EC001F0060ED89000360136E82EFBD759
:1037A000C00E0024E8CF4DF0FF0E0120E8CF4EF010
:1037B00036A60DD0FF0E026803684DC000F04EC063
:1037C00001F0DCEC2FF004C04DF005C04EF03F845A
:1037D000120032C000F0070E00160004D8A4120038
:1037E0003338E842070B300FD96E8098D95000016A
:1037F000B86F4D0E29EC12F080881200D950000FDE
:1038000010E6E30F0EE71D0F020D080EF324F66E0F
:10381000050EF420F76E0900F5500900F5CFFAFF08
:10382000F96E120030501F0B0001B26FB36BB25132
:10383000B36F31C0B2F0B211D8B41200400EB2155D
:10384000F36EF46A3F0EB2C000F0B3C001F0001690
:10385000016AD890B331036EB231026EC00BF66EBE
:103860000350F76E0050F610B26F0150F710B36FAF
:10387000F450F310D8A41200B2A92ED00F0EB2C08B
:1038800000F0B3C001F00016016AD890B331036EA6
:10389000B231026EF00BF66E0350F76E0050F61068
:1038A000B26F0150F710B36F190E026E036AB2C007
:1038B00000F0B3C001F0DCEC2FF0180E0424E8CFC8
:1038C00067F0FC0E0520E8CF68F0000EE8CF69F045
:1038D000E8CF6AF03E861200B2C0B8F0B3C0B9F0CB
:1038E0006EEC15F000C0B0F001C0B1F00001B151B4
:1038F000B011D8B41200640E046E056A066A076A35
:10390000B0C000F0B1C001F0000E01BEFF0E026EAB
:10391000036E6BEC2EF000C067F001C068F002C0CF
:1039200069F003C06AF00001B40E6727FB0E68233C
:10393000FF0E69236A233E86120030501F0BF36E80
:10394000F46AF350F46E31C0F3FFF450F310D8B4BE
:1039500012000001476B486BF4A802D0100E471309
:10396000F4A603D00001100E4813F4A403D0000104
:10397000200E4713F4A203D00001200E4813F4A038
:1039800003D00001400E4713F3AE03D00001400EF8
:103990004813F3AA03D00001010E4813F3A803D083
:1039A0000001010E4713F3A603D00001020E4813D5
:1039B000F3A403D00001020E4713F3A203D00001C9
:1039C000040E4813F3A003D00001040E47136CEC5F
:1039D00013F011D0310E05D0340E03D0350E01D0C6
:1039E000380ED96E8098D9500001B86F530E29EC6B
:1039F00012F0808816D047C002F048C003F00CD007
:103A000002504C0AEBE0FC0AE7E00BD00250140A2B
:103A1000E1E0750AE5E005D003501D0AF1E0030A74
:103A2000F5E03E8E120003C1E8FF000A01E1FAD67C
:103A3000040A01E1F7D6010A80E0150A01E1F2D695
:103A4000010A02E1C5EF18F0030A02E1B5EF18F030
:103A5000060A01E1E7D6010A01E16FD71200FBEC8B
:103A600001F0180EA96E3F0EA616A680A8A002D0DF
:103A70003E8001D03E90FBEC01F0180EA96E3F0E87
:103A8000A616A680A8A202D03D8E01D03D9EFBECDA
:103A900001F0180EA96E3F0EA616A680A8A402D0AB
:103AA0003D8601D03D96FBEC01F0180EA96E3F0E4D
:103AB000A616A680A8A602D03D8A01D03D9AFBECAE
:103AC00001F0180EA96E3F0EA616A680A8A802D077
:103AD0003D8C01D03D9CFBEC01F0180EA96E3F0E11
:103AE000A616A680A8AA02D03D8801D03D98FBEC7E
:103AF00001F0190EA96E3F0EA616A680A8CF05F1FB
:103B00001200FBEC01F0190EA96E05C1A8FF3F0ED3
:103B1000A616D890F2BED880F29EA684550EA76E47
:103B2000AA0EA76EA682A198A694D8B0F28E120013
:103B30000001B06B3EB0B0813DAE02D00001B08359
:103B40003DA602D00001B0853DAA02D00001B08799
:103B50003DAC02D00001B0893DA802D00001B08B7D
:103B6000FBEC01F0180EA96E0001B051A86E3F0EDB
:103B7000A616D890F2BED880F29EA684550EA76EE7
:103B8000AA0EA76EA682A198A694D8B0F28E1200B3
:103B9000B86AAF6EAE6AAE6AAE6A1200FBEC01F0B4
:103BA0001A0EA96E3F0EA616A680A850F1D7FBEC00
:103BB00001F01B0EA96E3F0EA616A680A850C86E77
:103BC000280EC66EC56A9E96A1961200E8CFF2F343
:103BD000E9CFF1F3EACFF0F3D9CFEFF3DACFEEF399
:103BE00004C0EDF303C0ECF302C0EBF301C0EAF351
:103BF00000C0E9F3F4CFE8F3F3CFE7F39EB09DA064
:103C000007D09E900001972B000E982399239A23AA
:103C1000F2B4F2AA72D0F29400014B2B000E4C23A6
:103C200081A66BD00F0E4BC000F04CC001F0001607
:103C3000016A01500010D8A460D006C1D9FF40D05D
:103C4000D9500B0D110EF324E8CF51F0010EF420E2
:103C5000E8CF52F0000100EE04F05151E926525134
:103C6000EA22EECF02F0EDCF03F04BC000F04CC0E3
:103C700001F00350015C02E10250005CD8A01FD0AB
:103C800000EE04F05151E9265251EA22EE6AED6A43
:103C900051C0E9FF52C0EAFFEE6AEE6AEE6AED6AD1
:103CA00000EE08F05151E9265251EA22EE6AED6A1F
:103CB00000EE0AF05151E9265251EA22EF6AD92A60
:103CC000100E06C102F0036A0226000E0322D9CFAD
:103CD00000F0016A0150800A046E0350800A045CFF
:103CE00002E10250005C410ED8B002D0D964A8D7DE
:103CF000D96401D0D96AD9CF06F19EBA9DAA0AD05B
:103D0000AE50156EABB202D0ABA402D0AB98AB886C
:103D1000010E166EE7C3F3FFE8C3F4FFE9C300F03A
:103D2000EAC301F0EBC302F0ECC303F0EDC304F00F
:103D3000EEC3DAFFEFC3D9FFF0C3EAFFF1C3E9FF37
:103D4000F2C3E8FF3CC0E0FFF3C3D8FF1000D06A25
:103D5000200E9D6EF06AF16AC00EF26E896A80884C
:103D60000F0E926E8A6AFC0E936E8B6AC10E946E71
:103D7000010EC26E0E0EC16EBE0EC06E010EE8CFF9
:103D800000F1FBEC01F0090EA96E3F0EA616A6800D
:103D9000A850420AD8A460D0FBEC01F00A0EA96E2C
:103DA0003F0EA616A680000EA6B0010E006E016A98
:103DB000A8502E0AD8A450D0FBEC01F00B0EA96E2F
:103DC0003F0EA616A680000EA6B0010E006E016A78
:103DD000A850560AD8A440D0FBEC01F00C0EA96EF6
:103DE0003F0EA616A680000EA6B0010E006E016A58
:103DF000A850450AD8A430D0FBEC01F00D0EA96EF6
:103E00003F0EA616A680000EA6B0010E006E016A37
:103E1000A8504C0AD8A420D0FBEC01F00E0EA96EDD
:103E20003F0EA616A680000EA6B0010E006E016A17
:103E3000A8504C0AD8A410D0FBEC01F00F0EA96ECC
:103E40003F0EA616A680000EA6B0010E006E016AF7
:103E5000A850450AD8B402D00101006B800EC76E8D
:103E6000A6DE8098240EAC6E900EAB6E81A803D0B7
:103E7000190E8EDE02D0020E8BDE80883D90166A0F
:103E80003E82EDDD08EC27F046EC12F06DEC0FF011
:103E9000809840EC04F08088809854EC10F0808882
:103EA000700E0001B06F6E0EB16F6F0E99EC14F0D2
:103EB00080A23AD0040EE8CF05F123DE520E44EC86
:103EC00009F0590E44EC09F0520E44EC09F0590E79
:103ED00044EC09F00D0E44EC09F00A0E44EC09F034
:103EE0000001AF0EB76F000EB86F36EC09F0D8A026
:103EF000F7D70001AF513F0AD8A403D054EC10F01B
:103F000004D00001AF5144EC09F08098FA0E000192
:103F1000AF6F80880001AF07AF29D8B4C9D7640E4E
:103F2000196E1DEC27F0F6D7810ECD6E9E90CE6AED
:103F3000CF6A05C1E8FF040AD8A402D09D8001D051
:103F40009D90870ED56E000EE8CF06F1000106C1E8
:103F50004BF04C6B4BC0D6FF4CC0D7FF808835EC84
:103F600021F082A487D01450D8B405D0262A000EA0
:103F700027222822292205C1E8FF020AD8B40FD03F
:103F800005C1E8FF030AD8B40AD005C1E8FF080A52
:103F9000D8B405D005C1E8FF040AD8A404D0020EA5
:103FA000E8CF01F148D0000EC2B2010E006EC2503F
:103FB0000014D8A404D0C3CF45F0C4CF46F02E38A7
:103FC000E8461F0BE8CF03F12E50070BE8CF02F1B4
:103FD00053EC17F081A603D082EC16F003D0020E4A
:103FE000E8CF01F13DBA3EA423D053C000F054C045
:103FF00001F055C002F056C003F0046A056A066A73
:104000000350076E0750041005100610D8A410D0F6
:1040100000EE63F000015351EE1808E15451EE1820
:1040200005E15551EE1802E15651EE18D8A497D784
:104030003EB0A6EC18F03EA217D080A203D03BEC15
:1040400011F017D081A405D081A413D01450D8B496
:1040500010D081A606D081A60CD001010153D8B49E
:1040600008D03DEC0BF005D01E2A000E1F222022A6
:10407000212282940001AF0EB76F000EB86F36ECAC
:1040800009F0D8B07AD0D1D03E82CFD03E92CDD0F8
:1040900054EC10F0CAD061EC10F0C7D058D65DECEB
:1040A0000EF0C3D037EC0FF0C0D008EC27F0BDD035
:1040B0003BEC11F0BAD046EC12F0B7D096EC11F010
:1040C000B4D098EC0FF0B1D0D1EC0FF0AED0AEEC94
:1040D0000FF0ABD0AEEC0FF0A8D03D9629DDA5D007
:1040E0003D8626DDA2D03D9A23DD9FD03D8A20DD8E
:1040F0009CD03E901DDD99D03E801ADD96D03D9E2D
:1041000017DD93D03D8E14DD90D03D9C11DD8DD018
:104110003D8C0EDD8AD03D980BDD87D03D8808DDD3
:1041200084D096EC13F081D04CEC14F07ED00101D9
:10413000056BE7DC20D0010EE8CF05F1E2DC1BD0F7
:10414000020EE8CF05F1DDDC16D0030EE8CF05F155
:10415000D8DC11D0040EE8CF05F1D3DCCE6ACF6AEB
:104160009D8063D0080EE8CF05F1CBDC04D0090EAA
:10417000E8CF05F1C6DC9D9058D00001AF51110A7F
:1041800083E0020A83E0230AD2E0010AD4E0030AB2
:10419000D7E0010ADAE0070ADDE00C0AE3E0010AF1
:1041A000E6E0060A01E174D77E0A97E0020A83E09E
:1041B000070AB1E0010A85E0030A95E00F0A87E0EB
:1041C000050AA3E01C0A01E16AD7020A01E166D7E9
:1041D000010A01E16AD7070AA4E0030A90E00F0A86
:1041E00088E0390A01E17CD7020A01E167D7070AB2
:1041F00095E0010A01E168D7030A01E177D70F0AC8
:1042000001E168D7050A84E0030A01E144D71F0AE7
:1042100001E148D7030A01E14BD7070A85E0030A09
:1042200001E170D70F0A01E167D73DA002D0010E6E
:1042300001D0000E006E81A602D0010E01D0000E4A
:10424000001AD8B48CD6F294F29A81B6F28A3D90D4
:1042500081B63D8084D6F28E222B000E23232423A8
:104260002523D8B008EC27F001D0F28E829216B147
:104270001200F29E82B082A0F8D700F016B11200B0
:1042800082A082B0FBD7CE50186F00F082B082A01F
:10429000ECD700F000F000F082A082B0EFD700F081
:1042A00000F000F082A082B0E9D700F000F000F04A
:1042B00082A082B0E3D700F000F000F082A082B0CC
:1042C000DDD700F000F000F082B082A0CED700F081
:1042D00000F000F082A082B0D1D700F000F000F032
:1042E00082B082A0C2D700F000F000F082A082B0BD
:1042F000C5D700F000F000F082A082B0BFD700F078
:1043000000F000F082A082B0B9D700F000F000F019
:1043100082A082B0B3D700F000F000F082A082B09B
:10432000ADD700F000F000F082A082B0A7D7829451
:10433000828200F082302E37146B2EB1142B00F0E5
:1043400082502E19010B87E000F000F082302E37EA
:1043500000F000F000F000F082502E19010B01E196
:104360007AD700F082302E3700F000F000F000F035
:1043700082502E19010B01E16ED700F082302E37EA
:1043800000F000F000F000F082502E19010B01E166
:1043900062D700F082302E3700F000F000F000F01D
:1043A00082502E19010B01E156D700F082302E37D2
:1043B00000F000F000F000F082502E19010B01E136
:1043C0004AD700F082302E3700F000F000F000F005
:1043D00082502E19010B01E13ED700F082302E37BA
:1043E00000F000F000F0C28282502E19010B01E1B2
:1043F00032D700F082302F3700F000F000F000F0EC
:1044000082502F19010B01E126D700F082302F379F
:1044100000F000F000F000F082502F19010B01E1D4
:104420001AD700F082302F3700F000F000F000F0D3
:1044300082502F19010B01E10ED700F082302F3787
:1044400000F000F000F000F082502F19010B01E1A4
:1044500002D700F082302F3700F000F000F000F0BB
:1044600082502F19010B01E1F6D600F082302F3770
:1044700000F000F000F000F082502F19010B01E174
:10448000EAD600F082302F3700F000F000F000F0A4
:1044900082502F19010B01E1DED600F082302F3758
:1044A00000F000F000F000F082502F19010B01E144
:1044B000D2D600F08230303700F000F000F000F08B
:1044C00082503019010B01E1C6D600F0823030373E
:1044D00000F000F000F000F082503019010B01E113
:1044E000BAD600F08230303700F000F000F000F073
:1044F00082503019010B01E1AED600F08230303726
:1045000000F000F000F000F082503019010B01E1E2
:10451000A2D600F08230303700F000F000F000F05A
:1045200082503019010B01E196D600F0823030370D
:1045300000F000F000F000F082503019010B01E1B2
:104540008AD600F08230303700F000F000F000F042
:1045500082503019010B01E17ED600F082303037F5
:1045600000F000F000F000F082503019010B01E182
:1045700072D600F08230313700F000F000F000F029
:1045800082503119010B01E166D600F082303137DB
:1045900000F000F000F000F082503119010B01E151
:1045A0005AD600F08230313700F000F000F000F011
:1045B00082503119010B01E14ED600F082303137C3
:1045C00000F000F000F000F082503119010B01E121
:1045D00042D600F08230313700F000F000F000F0F9
:1045E00082503119010B01E136D600F082303137AB
:1045F00000F000F000F000F082503119010B01E1F1
:104600002AD600F08230313700F000F000F000F0E0
:1046100082503119010B01E11ED600F08230313792
:1046200000F000F000F000F082503119010B01E1C0
:1046300012D600F08230323700F000F000F000F0C7
:1046400082503219010B01E106D600F08230323778
:1046500000F000F000F000F082503219010B01E18F
:10466000FAD500F08230323700F000F000F000F0B0
:1046700082503219010B01E1EED500F08230323761
:1046800000F000F000F000F082503219010B01E15F
:10469000E2D500F08230323700F000F000F000F098
:1046A00082503219010B01E1D6D500F08230323749
:1046B00000F000F000F000F082503219010B01E12F
:1046C000CAD500F08230323700F000F000F000F080
:1046D00082503219010B01E1BED500F08230323731
:1046E00000F000F000F000F082503219010B01E1FF
:1046F000B2D500F08230333700F000F000F000F067
:1047000082503319010B01E1A6D500F08230333716
:1047100000F000F000F000F082503319010B01E1CD
:104720009AD500F08230333700F000F000F000F04E
:1047300082503319010B01E18ED500F082303337FE
:1047400000F000F000F000F082503319010B01E19D
:1047500082D500F08230333700F000F000F000F036
:1047600082503319010B01E176D500F082303337E6
:1047700000F000F000F000F082503319010B01E16D
:104780006AD500F08230333700F000F000F000F01E
:1047900082503319010B01E15ED500F082303337CE
:1047A00000F000F000F000F082503319010B01E13D
:1047B00052D500F08230343700F000F000F000F005
:1047C00082503419010B01E146D500F082303437B4
:1047D00000F000F000F000F082503419010B01E10C
:1047E0003AD500F08230343700F000F000F000F0ED
:1047F00082503419010B01E12ED500F0823034379C
:1048000000F000F000F000F082503419010B01E1DB
:1048100022D500F08230343700F000F000F000F0D4
:1048200082503419010B01E116D500F08230343783
:1048300000F000F000F000F082503419010B01E1AB
:104840000AD500F08230343700F000F000F000F0BC
:1048500082503419010B01E1FED400F0823034376C
:1048600000F000F000F000F082503419010B01E17B
:10487000F2D414A1C2D28230353700F000F000F03B
:1048800082503519010B01E1E6D400F08230353752
:1048900000F000F000F000F082503519010B01E14A
:1048A000DAD400F08230353700F000F000F000F08C
:1048B00082503519010B01E1CED400F0823035373A
:1048C00000F000F000F000F082503519010B01E11A
:1048D000C2D400F08230353700F000F000F000F074
:1048E00082503519010B01E1B6D400F08230353722
:1048F00000F000F000F000F082503519010B01E1EA
:10490000AAD400F08230353700F000F000F000F05B
:1049100082503519010B01E19ED400F08230353709
:1049200000F000F000F000F082503519010B01E1B9
:1049300092D400F08230363700F000F000F000F042
:1049400082503619010B01E186D400F082303637EF
:1049500000F000F000F000F082503619010B01E188
:104960007AD400F08230363700F000F000F000F02A
:1049700082503619010B01E16ED400F082303637D7
:1049800000F000F000F000F082503619010B01E158
:1049900062D400F08230363700F000F000F000F012
:1049A00082503619010B01E156D400F082303637BF
:1049B00000F000F000F000F082503619010B01E128
:1049C0004AD400F08230363700F000F000F000F0FA
:1049D00082503619010B01E13ED400F082303637A7
:1049E00000F000F000F000F082503619010B01E1F8
:1049F00032D400F08230373700F000F000F000F0E1
:104A000082503719010B01E126D400F0823037378C
:104A100000F000F000F000F082503719010B01E1C6
:104A20001AD400F08230373700F000F000F000F0C8
:104A300082503719010B01E10ED400F08230373774
:104A400000F000F000F000F082503719010B01E196
:104A500002D400F08230373700F000F000F000F0B0
:104A600082503719010B02E12BEF21F000F0823068
:104A7000373700F000F000F000F082503719010BDA
:104A800002E12BEF21F000F08230373700F000F028
:104A900000F000F082503719010B02E12BEF21F0FA
:104AA00000F08230373700F000F000F000F0825064
:104AB0003719010B02E12BEF21F000F0823038377B
:104AC00000F000F000F000F082503819010B02E114
:104AD0002BEF21F000F08230383700F000F000F0CA
:104AE00000F082503819010B02E12BEF21F000F0A9
:104AF0008230383700F000F000F000F082503819B2
:104B0000010B02E12BEF21F000F08230383700F08A
:104B100000F000F000F082503819010B02E12BEF99
:104B200021F000F08230383700F000F000F000F0A3
:104B300082503819010B02E12BEF21F000F0823096
:104B4000383700F000F000F000F082503819010B07
:104B500002E12BEF21F000F08230383700F000F056
:104B600000F000F082503819010B02E12BEF21F028
:104B700000F08230383700F000F000F000F0825092
:104B80003819010B02E12BEF21F000F082303937A8
:104B900000F000F000F000F082503919010B02E142
:104BA0002BEF21F000F08230393700F000F000F0F8
:104BB00000F082503919010B02E12BEF21F000F0D7
:104BC0008230393700F000F000F000F082503919DF
:104BD000010B02E12BEF21F000F08230393700F0B9
:104BE00000F000F000F082503919010B02E12BEFC8
:104BF00021F000F08230393700F000F000F000F0D2
:104C000082503919010B02E12BEF21F000F08230C4
:104C1000393700F000F000F000F082503919010B34
:104C200002E12BEF21F000F08230393700F000F084
:104C300000F000F082503919010B02E12BEF21F056
:104C400000F08230393700F000F000F000F08250C0
:104C50003919010B02E12BEF21F000F082303A37D5
:104C600000F000F000F000F082503A19010B02E170
:104C70002BEF21F000F082303A3700F000F000F026
:104C800000F082503A19010B02E12BEF21F000F005
:104C900082303A3700F000F000F000F082503A190C
:104CA000010B02E12BEF21F000F082303A3700F0E7
:104CB00000F000F000F082503A19010B02E12BEFF6
:104CC00021F000F082303A3700F000F000F000F000
:104CD00082503A19010B02E12BEF21F000F08230F3
:104CE0003A3700F000F000F000F082503A19010B62
:104CF00002E12BEF21F000F082303A3700F000F0B3
:104D000000F000F082503A19010B02E12BEF21F084
:104D100000F082303A3700F000F000F000F08250EE
:104D20003A19010B02E12BEF21F000F082303B3702
:104D300000F000F000F000F082503B19010B02E19E
:104D40002BEF21F000F082303B3700F000F000F054
:104D500000F082503B19010B02E12BEF21F000F033
:104D600082303B3700F000F000F000F082503B1939
:104D7000010B02E12BEF21F000F082303B3700F015
:104D800000F000F000F082503B19010B02E12BEF24
:104D900021F000F082303B3700F000F000F000F02E
:104DA00082503B19010B02E12BEF21F000F0823021
:104DB0003B3700F000F000F000F082503B19010B8F
:104DC00002E12BEF21F000F082303B3700F000F0E1
:104DD00000F000F082503B19010B02E12BEF21F0B3
:104DE00000F082303B3700F000F000F000F082501D
:104DF0003B19010B02E12BEF21F0829282842A2BD6
:104E0000000E2B232C232D23D8B002D8F28E1200B3
:104E1000226B236B246B256B1A6B1B6B1C6B1D6B3E
:104E2000266B276B286B296B2A6B2B6B2C6B2D6BDE
:104E30001E6B1F6B206B216B1200827200F082745C
:104E4000192FFBD71200E96AEA6AF86A0001D890C4
:104E5000023603360232063607360632F6CF11F036
:104E6000F7CF12F00C6AE86A076440EF2FF0036492
:104E700049EF2FF0025006180F6E028E068E000EBC
:104E8000F76ED89006344C0FF66ED8B0F72A0900AA
:104E9000F5CF0EF00900F5CF10F00900F5CF08F0BE
:104EA0000900F5CF09F008500E5C086E0950105843
:104EB000096E08500D6E0402F4CFF7FF0950050289
:104EC000F4CF09F0F3CF08F00402F350F726F450C2
:104ED0000822E86A09220D500502F350F726F45023
:104EE0000822E86A09220D6AF7500D5E08500E5A32
:104EF0000950105A02C008F001C0F7FF00C0F6FFC9
:104F000000500D02F4CF09F001500E02F4CF00F072
:104F1000F3CF0AF00D02F3500926F4500A22E86A92
:104F20000022F6500E02F3500926F4500A22E86AD5
:104F3000002202510D02F3500A26F45000220251C1
:104F40000E02016AE86A0122F3500026F4500122A1
:104F5000F6501002F3500A26F4500022026AE86A62
:104F600001220222F7501002F3500026F4500122D1
:104F7000E86A022208501002F3500126F45002227F
:104F800002BE05D00A360036013602360C0606503F
:104F9000086E05C0F7FF04C0F6FF04500D02F4CF01
:104FA00009F005500E02F4CF04F0F3CF0BF00D0220
:104FB000F3500926F4500B22E86A0422F6500E0240
:104FC000F3500926F4500B22E86A042206500D0221
:104FD000F3500B26F450042206500E02056AE86ACC
:104FE0000522F3500426F4500522F6501002F35027
:104FF0000B26F4500422066AE86A05220622F750BE
:105000001002F3500426F4500522E86A06220850E4
:105010001002F3500526F450062206AE06BC06D058
:1050200009360B360436053606360C2A0B1E041ECE
:10503000051E061E0B2AE86A04220522062202C06B
:1050400010F001C00EF000C00DF00AC0F6FF0050D5
:105050000402F4CF09F001500B02F450092601506C
:1050600004020A6AE86A0A22F3500926F4500A2266
:10507000F6500502F4500926006AE86A0A22002266
:105080000D500502F3500926F4500A22E86A002266
:105090000E500502F3500A26F4500022025004027A
:1050A000F3500A26F450002202500502016AE86A11
:1050B0000122F3500026F450012210500B02F3504D
:1050C0000926F4500A22E86A002201221050060242
:1050D000F4CF02F0F3500126E86A0222F6500602ED
:1050E000F3500926F4500A22E86A00220122022223
:1050F0000D500602F3500A26F4500022E86A0122FD
:1051000002220E500602F3500026F4500122E86AF3
:10511000022202BE0CD00A360036013602360C06D8
:1051200002BE05D00A360036013602360C0607509C
:10513000035E800ED8A00AD00C24032611C0F6FF0F
:1051400012C0F7FFD8B031EF2FF009D00C2403269E
:1051500011C0F6FF12C0F7FFD8A036EF2FF00AAE4D
:1051600014D0D880800E0A640030E86A0022012240
:105170000222D8A00AD002320132003211C0F6FF5A
:1051800012C0F7FF034A31EF2FF00FAE029E11C09D
:10519000F6FF12C0F7FF023603320232D0EF2FF0D3
:1051A000D500D5C004F0D6C005F0D7C006F0D8C0F1
:1051B00007F0000E006A016A026A036A50EC2FF0E1
:1051C000D8A006D0000E006A016A026A036A1200C3
:1051D000D5C0DFF0D6C0E0F0D7C0E1F0D8C0E2F033
:1051E000046A056A800E066E3F0E076EDFC000F08F
:1051F000E0C001F0E1C002F0E2C003F050EC2FF09B
:10520000D8B018D0DFC004F0E0C005F0E1C006F06F
:10521000E2C007F0006A016A800E026E3F0E036E64
:1052200023EC27F000C0DFF001C0E0F002C0E1F0A5
:1052300003C0E2F0DFC0E3F0E0C0E4F0E1C0E5F07D
:10524000E2C0E6F00001D90EE76F000EE86F8BECCC
:105250002FF000C0DFF001C0E0F002C0E1F003C0B9
:10526000E2F0DFC0E3F0E0C0E4F0E1C0E5F0E2C06E
:10527000E6F0020E026E036AD9C000F0DAC001F057
:10528000A6EC2FF004C0E7F005C0E8F0E1EC2EF04A
:1052900000C0DFF001C0E0F002C0E1F003C0E2F0C6
:1052A000046A056A800E066E3F0E076ED5C000F0D8
:1052B000D6C001F0D7C002F0D8C003F050EC2FF0F8
:1052C000D8B018D0DFC004F0E0C005F0E1C006F0AF
:1052D000E2C007F0006A016A800E026E3F0E036EA4
:1052E00023EC27F000C0DFF001C0E0F002C0E1F0E5
:1052F00003C0E2F0140EF66EF76ADFC004F0E0C0FF
:1053000005F0E1C006F0E2C007F0D5C000F0D6C05D
:1053100001F0D7C002F0D8C003F023EC27F0DFC0C3
:1053200004F0E0C005F0E1C006F0E2C007F001ECD7
:105330002EF0046A056A066A400E076E23EC27F019
:1053400000C0DBF001C0DCF002C0DDF003C0DEF025
:105350000001E251DE1908E1E151DD1905E1E051FA
:10536000DC1902E1DF51DB19D8B413D0DBC0DFF068
:10537000DCC0E0F0DDC0E1F0DEC0E2F0F60EE96E88
:105380000F0EEA6EEE06000EED5AEE50ED10D8A4A8
:10539000B4D7DFC000F0E0C001F0E1C002F0E2C02D
:1053A00003F01200CD00CDC000F0CEC001F0CFC0A0
:1053B00002F0D0C003F002EC00F000C004F001C025
:1053C00005F002C006F003C007F0006A016A800E13
:1053D000026E3F0E036E50EC2FF0000E006A016A61
:1053E000D8B003D0026A036A1200800E026E3F0E2C
:1053F000036ECDC004F0CEC005F0CFC006F0D0C023
:1054000007F0CDC000F0CEC001F0CFC002F0D0C098
:1054100003F0CEEC2CF000C004F001C005F002C097
:1054200006F003C007F0006A016A800E026E3F0EAC
:10543000036EFFEC2DF000C0D5F001C0D6F002C025
:10544000D7F003C0D8F0D1EC28F000C0D1F001C0F3
:10545000D2F002C0D3F003C0D4F0CDC000F0CEC073
:1054600001F0CFC002F0D0C003F002EC00F08F0ECC
:10547000046EC20E056E350E066E3F0E076E50ECC2
:105480002FF0D8B01CD0D1C004F0D2C005F0D3C0EA
:1054900006F0D4C007F0CDC000F0CEC001F0CFC000
:1054A00002F0D0C003F023EC27F000C0E1F001C00F
:1054B000E2F002C0E3F003C0E4F0B3EF2AF0000131
:1054C000CDC004F0CEC005F0CFC006F0D0C007F0CC
:1054D000D1C000F0D2C001F0D3C002F0D4C003F0BC
:1054E000D0AF22D04EEC30F023EC27F000C0E1F03A
:1054F00001C0E2F002C0E3F003C0E4F0B3EC2AF034
:1055000000C004F001C005F002C006F003C007F0BF
:10551000DB0E006E0F0E016EC90E026E3F0E036EA3
:10552000FFEC2DF04EEF30F023EC27F000C0E1F05F
:1055300001C0E2F002C0E3F003C0E4F0B3EC2AF0F3
:1055400000C004F001C005F002C006F003C007F07F
:10555000DB0E006E0F0E016EC90E026E3F0E036E63
:10556000FFEF2DF0E100E1C000F0E2C001F0E3C088
:1055700002F0E4C003F002EC00F000C0EAF001C069
:10558000EBF002C0ECF003C0EDF0EA0EE96E000EA5
:10559000EA6EEE50EE10EE10EE10D8A406D0000E1B
:1055A000006A016A026A036A1200EAC004F0EBC0F2
:1055B00005F0ECC006F0EDC007F0006A016A800E4D
:1055C000026E3F0E036E50EC2FF0000ED8A0010EBD
:1055D0000001E56FE551EAC004F0EBC005F0ECC056
:1055E00006F0EDC007F0D8B418D0006A016A800E4A
:1055F000026E3F0E036E23EC27F000C0EAF001C0FC
:10560000EBF002C0ECF003C0EDF0EAC004F0EBC038
:1056100005F0ECC006F0EDC007F0EAC000F0EBC00A
:1056200001F0ECC002F0EDC003F0CEEC2CF000C0B5
:10563000E6F001C0E7F002C0E8F003C0E9F0E6C020
:10564000F2F0E7C0F3F0E8C0F4F0E9C0F5F00001D3
:105650005A0EF66F050EF76F040EF86FF96B3EECFD
:105660002CF000C0EEF001C0EFF002C0F0F003C07B
:10567000F1F0E6C0F2F0E7C0F3F0E8C0F4F0E9C002
:10568000F5F00001420EF66F050EF76F050EF86F8C
:10569000F96B3EEC2CF0EEC004F0EFC005F0F0C06A
:1056A00006F0F1C007F023EC27F000C004F001C0C1
:1056B00005F002C006F003C007F0EA0EE96E000E26
:1056C000EA6E3CEC30F00001E551D8B41AD0EAC0E3
:1056D00004F0EBC005F0ECC006F0EDC007F0DB0E07
:1056E000006E0F0E016EC90E026E3F0E036EFFECD0
:1056F0002DF000C0EAF001C0EBF002C0ECF003C0F6
:10570000EDF00001EAC000F0EBC001F0ECC002F0E7
:10571000EDC003F0E4AF12004EEF30F0D100D1C085
:1057200000F0D2C001F0D3C002F0D4C003F002EC0C
:1057300000F000C0DDF001C0DEF002C0DFF003C009
:10574000E0F0D5C000F0D6C001F0D7C002F0D8C05C
:1057500003F002EC00F0DDC004F0DEC005F0DFC0B5
:1057600006F0E0C007F050EC2FF0D8A043D0D5C031
:1057700004F0D6C005F0D7C006F0D8C007F0D1C0FD
:1057800000F0D2C001F0D3C002F0D4C003F023EC8B
:1057900027F000C0E1F001C0E2F002C0E3F003C076
:1057A000E4F0B3EC2AF000C0D9F001C0DAF002C096
:1057B000DBF003C0DCF00001D8AF13D0DB0E046EC9
:1057C0000F0E056E490E066E400E076ED90EE96E7D
:1057D000000EEA6ED4BF03D008EC30F002D006EC25
:1057E00030F0D9C000F0DAC001F0DBC002F0DCC05C
:1057F00003F01200D1C004F0D2C005F0D3C006F00F
:10580000D4C007F0D5C000F0D6C001F0D7C002F078
:10581000D8C003F023EC27F000C0E1F001C0E2F0B3
:1058200002C0E3F003C0E4F0B3EC2AF04EEC30F039
:1058300000C0D9F001C0DAF002C0DBF003C0DCF038
:105840000001DB0E046E0F0E056EC90E066E3F0ED4
:10585000076ED90EE96E000EEA6ED4AF03D006ECE7
:1058600030F002D008EC30F0D9C000F0DAC001F01E
:10587000DBC002F0DCC003F01200F200F8C000F060
:10588000F9C001F0D89000360136D89000360136C4
:105890000001F6510026F751012200C0F6FF01C0B9
:1058A000F7FF030EF7640DD00900F5CF00F00900F3
:1058B000F5CF01F00900F5CF02F00900F5CF03F0B4
:1058C0000CD0F6CFE9FFF7CFEAFFEECF00F0EECF36
:1058D00001F0EECF02F0EECF03F000C0FAF001C00D
:1058E000FBF002C0FCF003C0FDF00001F951F8111B
:1058F000D8B44BD0FAC004F0FBC005F0FCC006F0F1
:10590000FDC007F0F2C000F0F3C001F0F4C002F0F7
:10591000F5C003F0CEEC2CF0F80EE96E000EEA6E46
:10592000EE06000EED5AEECFFEF0EDCFFFF00001D7
:10593000D890FE37FF37D890FE37FF37F651FE2755
:10594000F751FF23FEC0F6FFFFC0F7FF030EF76419
:105950000DD00900F5CF04F00900F5CF05F00900DE
:10596000F5CF06F00900F5CF07F00CD0F6CFE9FF30
:10597000F7CFEAFFEECF04F0EECF05F0EECF06F062
:10598000EECF07F001EC2EF0A8D7FAC000F0FBC074
:1059900001F0FCC002F0FDC003F01200E96AEA6AFF
:1059A000D8900236033602320636073606320A6AC5
:1059B000E86A0762036449EF2FF0025006180F6E81
:1059C000075003267E0ED8A005D0035ED8B031EF75
:1059D0002FF004D0035ED8A036EF2FF0028E068E93
:1059E00002C010F001C00EF000C00DF00050040223
:1059F000F4CF09F001500502F4CF00F0F3CF0AF024
:105A00000402F3500926F4500A22E86A00220D50DD
:105A10000502F3500926F4500A22E86A00220250D7
:105A20000402F3500A26F450002202500502016AD3
:105A3000E86A0122F3500026F45001220D500602BC
:105A4000F3500A26F4500022026AE86A0122022278
:105A50000E500602F3500026F4500122E86A02229A
:105A600010500602F3500126F450022202BE08D064
:105A70000A360036013602360306D8B436EF2FF068
:105A80000AAE10D0D880800E0A640030E86A002286
:105A900001220222D8A006D0023201320032034A8B
:105AA00031EF2FF00FAE029E023603320232D0EFFA
:105AB0002FF0EA00820EF66EF768170EEAC000F0CB
:105AC000EBC001F0ECC002F0EDC003F01DEC30F0D3
:105AD0000050F624F36E000EF720F46EF4AE0ED0F4
:105AE0000001000E006A016AEDBF03D0026A036A7A
:105AF0001200800E026EBF0E036E1200000EF45CE8
:105B00001D0ED8B4F35CEAC000F0EBC001F0ECC0AD
:105B100002F0EDC003F0D8B012000AEC2FF0F8EC60
:105B20002FF000C0EEF001C0EFF002C0F0F003C0B3
:105B3000F1F0EEC004F0EFC005F0F0C006F0F1C0E7
:105B400007F0EAC000F0EBC001F0ECC002F0EDC0DD
:105B500003F050EC2FF0D8B010D0046A056A800E24
:105B6000066E3F0E076EEEC000F0EFC001F0F0C011
:105B700002F0F1C003F0FFEF2DF0EEC000F0EFC037
:105B800001F0F0C002F0F1C003F012000C500D5C07
:105B90001BE3E80F06E3026A016A006A0D500C6E0F
:105BA00012000C500D5CFCE0F80F08E3080E0C2608
:105BB0000150006E0250016E026AF3D703320232C6
:105BC000013200320C2AEDD70D500C5CE80F04E3D3
:105BD000066A056A046A12000D500C5CE1E0F80FD9
:105BE00008E3080E0D260550046E0650056E066A81
:105BF000F3D707320632053204320D2AEDD7800E74
:105C0000071AE96AEA6AB1EC01F0BFEC01F0BEDF05
:105C10000EB032EC30F00EA209D0041E051E061E96
:105C2000071E000E042A0522062207220450002621
:105C30000550012206500222075003220E6A03AECD
:105C4000D9EF01F032EC30F00E80D9EF01F0D9003D
:105C5000D9C004F0DAC005F0DBC006F0DCC007F004
:105C6000DB0E006E0F0E016E490E026E400E036ECB
:105C700050EC2FF0D8B013D0E40E046ECB0E056EAE
:105C8000960E066E400E076ED9C000F0DAC001F025
:105C9000DBC002F0DCC003F0FFEC2DF012D0D9C065
:105CA00004F0DAC005F0DBC006F0DCC007F0DB0E64
:105CB000006E0F0E016EC90E026E3F0E036E01ECF8
:105CC0002EF000C0DDF001C0DEF002C0DFF003C046
:105CD000E0F0A8EF00F0E96AEA6A0050086E0150AF
:105CE000096E02500A6E03500B6E026A036A085076
:105CF0000402F3CF00F0F4CF01F00502F3500126C7
:105D0000F450022209500402F3500126F4500222FA
:105D1000D8B0032A08500602F3500226F45003229A
:105D200009500502F3500226F45003220A500402DF
:105D3000F3500226F450032208500702F3500326C2
:105D400009500602F35003260A500502F3500326B9
:105D50000B500402F3500326D0EF2FF0066A046ABA
:105D6000056A0250031003E1006A016A000C1F0E6D
:105D70000612D890062A02360336FCE303320232BA
:105D80000250005C0350015804E3016E0250005EB3
:105D9000D88004360536062E06BAF0D706AE05D0F2
:105DA000041E042AD8B40506051E0450026E0550D0
:105DB000036E06AC000C001E002AD8B40106011EBA
:105DC000000C0001E535E635810FE727D8B0E82B58
:105DD000E8BEE807E835000EE8210DE1E7517F0F46
:105DE000E3C000F0E4C001F0036EE6370332E5459E
:105DF000026E02321200E8AF05D0006A016A026A40
:105E0000036A12000068016802680368029EE8AF36
:105E1000039E1200E96AEA6AB1EC01F0820E0C26D8
:105E20000CBEBAEF01F0E80E0C260CBE12D0200E0C
:105E30000C5CD8B0BAEF01F00C52D8B406D00C0606
:105E40000036013602360336F7D70EB032EC30F0AA
:105E50001200D89003320232013200320C3EF9D7E0
:105E6000F4D713820236033202320BD01384023687
:105E700003320232800E026E036A016A006A05D0A4
:105E8000138603680268016800680F360332D0EF9A
:105E90002FF0026A016A006A0A6A036AD0EF2FF0E3
:105EA00003500718800B04E0073407500109120063
:105EB000039E07507F0B035C0AE10650025C07E17A
:105EC0000550015C04E10450005CD8B412000734B2
:105ED000D8B0010A076E073002091200C900C9C014
:105EE000CDF0CAC0CEF0CBC0CFF0CCC0D0F0D3EC58
:105EF00029F000C004F001C005F002C006F003C0A4
:105F000007F0DB0E006E0F0E016EC90E026E3F0E23
:105F1000036EFFEF2DF00001E7C0E9FFE8C0EAFFE4
:105F2000E535E635EF6E7E0EEE5EEF6AD8A0EF0641
:105F3000E6357E0EE66FE633E59FE3C000F0E4C091
:105F400001F0E5C002F0E6C003F0000C066A01AE05
:105F500006D0001E004A0106011E068C068E035064
:105F6000800B061A03AEAFEF2EF0021E024A0306A4
:105F7000031EAFEF2EF0016A026A036A00AEF8EF6B
:105F80002FF0010602060306F8EF2FF00E6A016AF1
:105F9000026A036A04EF30F0036A026A016A006A67
:105FA000E950EA1008E003C0EDFF02C0EDFF01C0B8
:105FB000EDFF00C0EFFF000C02500002F3CF04F031
:105FC000F4CF05F00102F350052603500002F35010
:105FD00005261200026A036A01AEF8EF2FF00206EE
:105FE0000306F8EF2FF00E6A026A036A04EF30F03E
:105FF0000E6A03AE03D00E8032EC30F0960E0C6EBB
:10600000E96AEA6AD9EF01F00E6AF8D7800E071A3A
:10601000EECF00F0EECF01F0EECF02F0EFCF03F0C5
:1060200003EF2EF0046E042A0406D8B4000CD890B6
:106030000036013602360336F7D7046E042A04060A
:10604000D8B4000CD8900332023201320032F7D7B4
:10605000EECF00F0EECF01F0EECF02F0EFCF03F085
:106060006DEF2EF0001E011E021E031E000E002A00
:106070000122022203221200EECF00F0EECF01F047
:10608000EECF02F0EFCF03F0D0EF2CF0EE6AEA5043
:10609000E262FCD7E950E162F9D71200023403341E
:0860A00002E0800E031A120059
:020000040030CA
:0E000000E33ED6FEFF7DBFFFFFFFFFFFFFFFC9
:0200000400F00A
:100000004144534220322E3920422E56454C4C4515
:1000100020284329323030391104197700000000BC
:10002000004A57EB00039F5BFFFFFFFFFFFFFFFF4F
:10003000FFFFFFFFFFFFFFFFFFFFFFFFFFFFFFFFD0
:10004000FFFFFFFFFFFFFFFFFFFFFFFFFFFFFFFFC0
:10005000FFFFFFFFFFFFFFFFFFFFFFFFFFFFFFFFB0
:10006000FFFFFFFFFFFFFFFFFFFFFFFFFFFF00009E
:100070000000000000000000000000000000000080
:020000040000FA
:00000001FF
